:020000040001F9
:1090000040330020C1930100C9930100CB930100BC
:10901000CD930100CF930100D19301000000000027
:10902000000000000000000000000000D3930100D9
:10903000D593010000000000D7930100D9930100EF
:1090400041970100DB930100B19A0100DB9301001D
:10905000DB9301000000000079950100DB93010023
:10906000DB930100DB930100DB930100DB93010044
:10907000DB930100DB930100DB930100DB93010034
:10908000DB93010099970100DB930100DB93010062
:10909000BD970100DB930100C1970100DB93010044
:1090A000DB930100DB9301000000000000000000E2
:1090B000DB930100DB9301000000000000000000D2
:1090C00000000000000000000000000000000000A0
:1090D0000000000000000000000000000000000090
:1090E0000000000000000000000000000000000080
:1090F0000000000000000000000000000000000070
:10910000000000000000000000000000000000005F
:10911000000000000000000000000000000000004F
:10912000000000000000000000000000000000003F
:10913000000000000000000000000000000000002F
:10914000000000000000000000000000000000001F
:10915000000000000000000000000000000000000F
:1091600000000000000000000000000000000000FF
:1091700000000000000000000000000000000000EF
:1091800000000000000000000000000000000000DF
:1091900000000000000000000000000000000000CF
:1091A00000000000000000000000000000000000BF
:1091B00000000000000000000000000000000000AF
:1091C000000000000000000000000000000000009F
:1091D000000000000000000000000000000000008F
:1091E000000000000000000000000000000000007F
:1091F000000000000000000000000000000000006F
:10920000DFF80CD000F07AF900480047DDD3010008
:109210004033002030B450E8012F93B2C489234476
:109220008489A34228BF1B1B0489A34202BFBFF34A
:109230002F8F002007E0C3EA020340E80134002C2E
:10924000E9D14FF001000A6030BC704750E8012FAF
:10925000C2EA024240E801210029F7D1704730B448
:1092600050E8022F1FFAA2F3C488A34202BFBFF343
:109270002F8F00200DE0C48923448489A34228BF96
:109280001B1BC2EA034340E80234002CE8D14FF034
:1092900001000A6030BC704750E8022FC2EA224247
:1092A00040E802210029F7D17047034653E8022F16
:1092B000D988B2EB324F4FF0000017BF92B241EAAB
:1092C000014142EA014104E05A68B2EB324F08BF63
:1092D000012043E80212002AE8D1704730B4044666
:1092E00054E8000F0D4644E80053002BF8D11560F8
:1092F00030BC704730B4044654E8000F40EA010522
:1093000044E80053002BF7D1156030BC704730B4EF
:10931000044654E8000F00EA010544E80053002B1E
:10932000F7D1156030BC704730B4044654E8000FE4
:1093300080EA010544E80053002BF7D1156030BCEA
:10934000704730B4044654E8000F00EB010544E8D0
:109350000053002BF7D1156030BC704730B4044681
:1093600054E8000FA0EB010544E80053002BF7D1AF
:10937000156030BC704770B404464FF0000054E8EC
:10938000006F0D68AE4207BF44E80023012044E8A7
:1093900000630E60002B1CBF0020F0E770BC70471C
:1093A00030B4044654E8000F88422CBF451A0546E5
:1093B00044E80053002BF5D1156030BC7047000025
:1093C0000648804706480047FEE7FEE7FEE7FEE75F
:1093D000FEE7FEE7FEE7FEE7FEE7FEE7C5970100D2
:1093E000019201002DE9F05F0546002092469B4660
:1093F00088460646814640241BE0284641464746AB
:10940000224600F06BF853465A46C01A914110D3D9
:1094100011461846224600F016F82D1A67EB01088F
:109420004F4622460120002100F00DF817EB0009FD
:109430004E41201EA4F10104DFDC484631462A4695
:109440004346BDE8F09F202A04DB203A00FA02F1EF
:10945000002070479140C2F1200320FA03F3194322
:109460009040704700487047CC2A020040EA010350
:109470009B0703D009E008C9121F08C0042AFAD2CA
:1094800003E011F8013B00F8013B521EF9D270478E
:10949000D2B201E000F8012B491EFBD27047002236
:1094A000F6E710B513460A4604461946FFF7F0FFE3
:1094B000204610BD421C10F8011B0029FBD1801A68
:1094C000704730B504460020034600E05B1C934221
:1094D00003D2E05CCD5C401BF8D030BD202A04DB19
:1094E000203A21FA02F00021704721FA02F3D0401D
:1094F000C2F120029140084319467047064C074DBF
:1095000006E0E06840F0010394E807009847103453
:10951000AC42F6D3FFF778FEAC310200CC3102004A
:1095200070B58C1810F8015B15F0070301D110F825
:10953000013B2A1106D110F8012B03E010F8016B52
:1095400001F8016B5B1EF9D12B0705D40023521ED5
:109550000DD401F8013BFAE710F8013BCB1A921C3D
:1095600003E013F8015B01F8015B521EF9D5A1423B
:10957000D8D3002070BD00002DE9F04700268AB046
:10958000DFF85091B0464FF48075012437460696B7
:10959000284604F09FFF38B1D9F80403204203D0D5
:1095A000284604F08DFF26432D1D64007F1CADB2BC
:1095B000082FEDD34FF4BE74204604F08BFF48B162
:1095C000204604F07DFF46F0004606AA0121002057
:1095D00004F062FF404D16F0FF0F15D00127002464
:1095E00037420DD009EB8401D1F81005D1F81015E0
:1095F000C0F3042055F82420C1F3014102B1904783
:109600007F00641C082CEBD3002E5FDA4FF0FF3094
:10961000CDF8108054E0281910F8507F90F9000020
:1096200027F0C008401C3BD007A9404604F0F1F9E0
:1096300010B34FEA9719404602F090F855F82070A1
:109640001FB1B9F1030F03D006E0B9F1030F27D121
:1096500004A9404604F0E5F94FF0A04101EB880071
:10966000D0F8000706A9C0F3014A404604F0D1F93A
:1096700018B1BAF1020F03D012E0BAF1030F0FD103
:10968000B9F1030F08D1BAF1020F1DD002214046F3
:1096900004F0E6FE761CF6B217B149464046B847DC
:1096A000641C042CB7D3002E10D06A460121002080
:1096B00004F0F2FE06990098884207D006900498BC
:1096C000002634460790A6E70321E0E70AB0BDE88C
:1096D000F087000000600040D422002000F01F024C
:1096E000012191404009800000F1E020C0F8801283
:1096F000704700F01F02012191404009800000F1F5
:10970000E020C0F80011704700F01F0201219140D5
:109710004009800000F1E020C0F8001270474907BE
:10972000090E002806DA00F00F0000F1E02080F8B2
:10973000141D704700F1E02080F80014704700000D
:1097400070B54FF48076304604F074FA114CB505CC
:1097500060B1304604F075FA0120C5F8080360795D
:1097600020B9012060712168002088474FF482767B
:10977000304604F05FFA00280AD0304604F061FA5F
:109780000220C5F808032168BDE8704001200847A1
:1097900070BD0000401C002007480021C0F84011A7
:1097A000C0F84411C0F84811C0F84C11C0F80011BD
:1097B000C0F8041108F0C0BA0010014008F00ABA5D
:1097C00005F0DCBBF0B5A848A74B012600781B1DAF
:1097D0001A1D4FF0805106280BD11C78240708D1A0
:1097E0001478C4F30314032C06D0042C04D0052CE5
:1097F00002D0062807D011E0B1F824439B4DC4F3F2
:1098000004242C6002E01C78240707D11478C4F3E8
:109810000314032C02D1974D954C6C67D1F830514D
:10982000D1F84442944FC4F342343C6006280CD132
:109830001C78240709D11478C4F30314032C04D131
:109840008E4C276827F0807727604FF080470024F0
:10985000C7F80C41C7F81041874F3F1F3C600628EE
:1098600007D11F783F0704D11778C7F30317032FD9
:1098700002D0062808D01FE0DFF8FCC103270CF156
:10988000640CCCF8007007E01F783F0714D11778FC
:10989000C7F30317032F0FD1DFF8E4C10527CCF876
:1098A0000070774F78373E60754F08373C600CF199
:1098B000040C3F27CCF80070724F3F68DFF8C8C136
:1098C000CCF800706F4F3F1D3F680CF1040CCCF8D2
:1098D00000706C4F08373F680CF1040CCCF8007036
:1098E000684F0C373F680CF1040CCCF80070654FE2
:1098F00010373F680CF1040CCCF80070614F14373E
:109900003F680CF1040CCCF800705E4F18373F68CC
:10991000DFF874C10CF1200CCCF80070594F1C37E3
:109920003F680CF1040CCCF80070564F20373F68AC
:109930000CF1040CCCF80070524F24373F680CF146
:10994000040CCCF800704F4F28373F680CF1040C22
:10995000CCF800704B4F2C373F680CF1040CCCF85E
:109960000070484F30373F68DFF81CC10CF1400CE5
:10997000CCF80070434F34373F680CF1040CCCF83E
:109980000070404F38373F680CF1040CCCF8007081
:109990003C4F3C373F680CF1040CCCF80070394F59
:1099A00040373F680CF1040CCCF80070DFF8DCC0E5
:1099B000FB27CCF80070062813D11F783F0710D181
:1099C0001778C7F30317032F03D0042F01D0052FF7
:1099D00007D1D1F85872DFF8B8C007F04F07CCF8BC
:1099E00000702C480268D20702D06FF001020260BA
:1099F000062D08D1D1F83401062804D12648016883
:109A000041F4806101604FF01021D1F8000200287C
:109A100003DBD1F80402002822DA204A166020482D
:109A20000368002BFCD01523C1F800320568002D17
:109A3000FCD0C1F8043201680029FCD01460016830
:109A40000029FCD0BFF34F8F0C48F0380168154A4D
:109A500001F4E06111430160BFF34F8F00BFFDE7E8
:109A6000124911480860F0BDE00F00F04035014098
:109A70000DF0ADBA00C007403C050040FCED00E031
:109A8000105600400404001020C5004018F50040A6
:109A9000E40E0040000400403C17004004E5014093
:109AA00000E401400400FA050090D003541D00209A
:109AB0000149024808F0C0B93023002000200040CE
:109AC00002E008C8121F08C1002AFAD17047704787
:109AD000002001E001C1121F002AFBD170470000E5
:109AE0000121202803DA81400548014003E0402895
:109AF00002DA2038814009B1012070470020704708
:109B0000FC06FFBD082806D228B1012803D004288E
:109B100001D0012070470020704710B560B159B1E5
:109B200002780B785208B2EB530F05D10622401C85
:109B3000491CFFF7C6FC08B1002010BD012010BD74
:109B4000800701D00020704701207047C3688B4216
:109B500006D811440069491E814201D8012070478E
:109B60000020704710B501220221002001F006FC00
:109B700008B1072810D107220221012001F0FEFBC5
:109B800008B1072808D100210A22084601F0F6FB97
:109B900008B1072800D1002010BD000000B5ABB00F
:109BA000AC216846FFF77BFC022101208DF80010F4
:109BB0008DF8020006228DF803200322ADF8102054
:109BC0000D4A05922822229244F250628DF87C00C0
:109BD0002392CDE927108DF898000848299069460E
:109BE000074800F036FC08B100F0ECF80121044809
:109BF00000F02CFC2BB000BD6C1B00201DF50100FB
:109C00002C1E002010B550B10A480321008801EB3A
:109C1000004009A104F044FE06F0ACFC03E003217F
:109C2000084800F0FDFC002803D0BDE8104000F01B
:109C3000C9B810BD9C1D0020457261736520626F1C
:109C40006E6473002C1E002070B58CB015460E4655
:109C500000236C46C3F10F01415CE1545B1C102BE7
:109C6000F8D30D2104F11000FFF719FC0020C0F11A
:109C70000F02315C2244401C11740328F7D368465C
:109C800046DF0020C0F10F01214491F82010295433
:109C9000401C0328F6D30CB070BD022001F078BA46
:109CA0000149097900F0F2BED01B002070B50024F4
:109CB000064D06E06868012110F8340005F038FA16
:109CC000641C28788442F5D3002070BD481C002015
:109CD000F8B515460C460646052A01D20720F8BD00
:109CE00005F022FB18B905F0E7FA0028F7D1124970
:109CF00000224E600C708D60C1E90422C1E9062289
:109D00000E4D0DE006EBC4002968009181788DF8B6
:109D1000011000780A4A694605F05CFA0028DED195
:109D2000641EE4B2EED2BDE8F84004480021054AC2
:109D3000001D00F053B80000481C0020502702000E
:109D400079C701008DBB010072B604F05FFE00BF51
:109D500004F096FC0028FBD1104C0121208801EB77
:109D600000400FA104F09CFD10480068C00700D01F
:109D700000BE2088022101EB00400DA104F090FDFF
:109D8000BFF34F8F0948E43801680D4A01F4E061E0
:109D900011430160BFF34F8F00BFFDE79C1D002002
:109DA000466174616C206572726F7200F0ED00E0C4
:109DB00053797374656D20726573657400000000DB
:109DC0000400FA050EB500210091CDE901106A46A4
:109DD00044F20100FFF7B8FF0EBD0000074B9B786F
:109DE00023B12AB120B10068037C1BB10820704761
:109DF000072070474174426100207047742300209F
:109E000070B506F0C7FF104800240B2104704470A1
:109E10000E4D817014206C602C706C70FFF75EFC2E
:109E200007211420FFF77BFC1420FFF762FC084891
:109E3000046007211120FFF772FC0548001F00682D
:109E4000A860002070BD000074230020681C002062
:109E5000081501402DE9FC47DFF8789099F80230A9
:109E600073B368B3052902D20720BDE8FC874369B4
:109E700033B3437C012B25D00027044600258846B8
:109E800016468DF80050684600F038F801A808F032
:109E90001FF9C8B1012101700F4944600968C0E988
:109EA0000218C0E904769DF8040089F801009DF8C5
:109EB000000000F047F81420FFF726FC2846D4E7FE
:109EC0000820D2E70F46D8E704259DF8000000F0EF
:109ED00039F8F3E774230020041501400649897816
:109EE00039B130B1416921B100210174022107F07B
:109EF000FFBE0820704700007423002030B5EFF348
:109F0000108172B60D4A9468012324B103700029B0
:109F100000D162B630BD93604FF0E023D3F880519A
:109F2000074C25401560C3F88041D3F88441546044
:109F30005A17C3F8842100220270E8E78024002029
:109F4000FC06FFBD0B498A68002A11D000280FD1FA
:109F5000EFF3108072B60B684FF0E022C2F80031C8
:109F60004B68C2F8043100228A60002800D162B632
:109F700070470000802400202DE9F0410646086863
:109F80000C46411C4FF0A0474FF0010506D005FAE2
:109F900000F1C7F80815206804F058FA6068411C01
:109FA00002D0002104F049FA3168A069C1F8240503
:109FB000607D217D32680843C2F86C05D4E9001247
:109FC0003068C0F80C15C0F81425207D012815D183
:109FD000A068411C02D0002104F02FFAE068411C67
:109FE00005D08540C7F80855E06804F02FFAD4E999
:109FF00002123068C0F80825C0F81015BDE8F081DD
:10A0000003F048B92DE9F047074600888EB0804636
:10A0100002F038FE824604462D4800252A46017883
:10A02000404600F04BFD7879400734D501254FF6C6
:10A03000FF7603AB2A460721504605F001FD0100DB
:10A0400004D0404607F09CF800252BE0B14631468D
:10A05000049802F06BFD064648450FD004460146C1
:10A06000404602F0F9FD4046FFF71AFE30B940467F
:10A0700007F058F84046FFF713FE48B12246072183
:10A08000504605F053FD010003D0404607F078F834
:10A0900000254E4506D0404605F0B6FE10B15046AC
:10A0A00002F0DCFD02208DF81800ADF81A807879F6
:10A0B000400701D5012000E002208DF820008DF836
:10A0C000215006A801F0D6FE0EB0BDE8F0870000D2
:10A0D000D01B00202DE9F0430546407C93B00E468E
:10A0E0000024A0B107949DF81C0020F00F00401C34
:10A0F00020F0F00010308DF81C00707B8DF81D00F2
:10A100009DF81E0020F00600801C8DF81E001C210A
:10A110006846FFF7C4F99DF8000040F002008DF892
:10A120000000697C11B140F0100001E020F0100047
:10A130008DF80000019403940494687C00B107A892
:10A14000CDE9050401278DF8427042F61920ADF8DB
:10A1500040000D94B07B8DF83400F07B8DF8350015
:10A160009DF83600142120F00600801C20F0190014
:10A170008DF83600307B8DF8440008A8FFF78FF982
:10A180000DF140080DF13409ADF8287011A8CDE9A2
:10A190000889ADF82A40ADF82C700C90A888AB1D4A
:10A1A00008AA6946AADF002838D1B06898B38DF8AC
:10A1B000427042F60810ADF840000D94307C8DF8E6
:10A1C00034009DF8350020F0FF008DF835009DF833
:10A1D000360020F00600801C20F019008DF83600B3
:10A1E0000EA8B16800F08DFF0646142108A8FFF7FD
:10A1F00056F9ADF828600EA8CDE90889ADF82A40D7
:10A20000ADF82C600C90E88805F10E0208A9ABDFD0
:10A21000002803D101E0FFE7EC81002013B0BDE886
:10A22000F083000010B50D490D4807F024F8C1B2C5
:10A230004FF6FE720B4800F0FBFA00280DD00828FC
:10A240000BD0132809D0112807D043F201418842CE
:10A2500003D0BDE81040FFF7B5BD10BDF01E0020D3
:10A260004C1B0020EC1D00200A4601461046AEDFC4
:10A2700070472DE9FC47002517880646158090F8A1
:10A280002D001446894630B13A462146484600F032
:10A290003FFC051E09D1B0784FF00C0A18B3208896
:10A2A000C846001DB84202D95046BDE8FC87684642
:10A2B00079DF0028F9D12088032108F800102088D0
:10A2C0001921401C80B2208008F800102088401C12
:10A2D00080B2208000EB0801BDF8000007F026FEE8
:10A2E000218808442080F0780222C8B1218896F99C
:10A2F000033001F1030C4846BC45D5D842542188AF
:10A300004FF0010C491C89B2218000F801C021885E
:10A31000491C89B2218009F801302088401C208026
:10A320007068B8B1218890F9003001F1030C4846FB
:10A33000BC45B9D8425421880A22491C89B22180DF
:10A3400042542188491C89B2218009F801302088B3
:10A35000401C2080308950B1CDE900474B46062291
:10A36000022106F1080007F0CBFE051E9DD1308AC0
:10A3700050B1CDE900474B460722032106F11000FA
:10A3800007F0BEFE051E90D1308B50B1CDE90047DD
:10A390004B461522142106F1180007F0B1FE051EE8
:10A3A00083D1306A30B13B462246494601F0E1FA9A
:10A3B000051EDBD1706A30B13B462246494603F0A8
:10A3C000E3F8051ED2D196F82C0038B13B46224660
:10A3D0004946304606F0E4FF051EC7D1307838B153
:10A3E0003B4622464946304603F054F9051EBDD18E
:10A3F00028465AE718B504460020ADF80000134679
:10A400006A46204600F006F8002802D0BDF8000099
:10A41000204418BD70B588B182B10024158803E0CE
:10A42000065D641C3444A4B2A54203D806197678AC
:10A430009E4201D08C42F3D38C4201D3002070BDE8
:10A44000A11C1180005D401E80B270BD80F83010EC
:10A4500070472DE9F0410D00044606D02CB195F867
:10A460007A000026012803D006E00E20BDE8F08126
:10A4700095F89800012829D0D5F8A000042825D007
:10A48000D5F89C00042821D04FF00108A6702C229A
:10A4900005F17801201DFEF7E9FF84F83060D5F85A
:10A4A000A4006063D5F8A800A0634FF6FF70A4F87D
:10A4B000A80004F19400C4F8A400C4F8AA60A4F8A9
:10A4C000AE6084F8B060207810B104E00720CDE7DA
:10A4D000FF2084F8540004F155011F27C4F894109C
:10A4E000A4F8987004F198022846FFF7C2FE0028ED
:10A4F000BCD115F13C0F0ED004F17401C4F89C10CE
:10A50000A4F8A07004F1A00205F13C00FFF7B1FE31
:10A510000028ABD103E0C4F89C60A4F8A06084F8E4
:10A520005180208BA4F8480084F83C80266484F88D
:10A53000506060696064454604F13C02002104F10A
:10A54000540072DF002891D125708FE710B5028882
:10A55000102A1BD0112A20D0262A1DD1007A0C46A1
:10A56000012801D0022817D1A0780521401CB0FB9A
:10A57000F1F201FB1201204600F052F800280BD046
:10A58000A16B002908D0BDE810400847C27B012A12
:10A5900002D18088A1F8A80010BD0C46002184F8E3
:10A5A000B2108088B4F8A8108842F5D1207900282C
:10A5B000F2D10121DFE710B50C46022801D00328B3
:10A5C00010D1607800280DD000206070A17820465E
:10A5D00000F026F8002805D0A16B002902D0BDE8C4
:10A5E0001040084710BD10B5044690F8540074DFC1
:10A5F000012084F8B200002084F8B40084F85000F0
:10A600000621204601F03CFE002808D1A178204612
:10A6100000F006F810B1A16B01B18847002010BD11
:10A620002DE9F05F044600780F4638B1A77000208E
:10A6300003F044FD012620B16670F4E00820BDE877
:10A64000F09F0025C4F8AA50A4F8AE5084F8B0508A
:10A65000A07910B1A078012806D0E07968B1A0787F
:10A66000012801D0022808D1616B21B184F8B160C2
:10A670000820884701E084F8B15004F1AB010020C4
:10A680000A5C0AB1304603E0401C0628F8D30020DB
:10A690004FF002084FF0030A4FF0040B012F06D0D1
:10A6A000022F0CD0032F0FD0042F15D110E0A17969
:10A6B00029B194F8241011B908B130460DE0E179C0
:10A6C00011B108B1404608E0207A08B1504604E0D4
:10A6D000607A08B1584600E02846A070616B41B12D
:10A6E000032801D0042804D1607910B194F8B20095
:10A6F000A0B184F8B35004F13C0018210746FEF7DE
:10A70000CEFE04F12C0084F83C60814605F072FC1A
:10A7100058B194F82C0084F8510008E084F8B45043
:10A7200084F8B36007208847E5E784F8516094F81F
:10A73000240050B1484605F05DFC20B194F8280093
:10A7400084F8520001E084F8526084F85050A278F6
:10A7500004F1AA0104F19409052A4DD2DFE802F0C0
:10A7600065030F1B320084F83160C4F8A450C4E9BB
:10A77000101584F83C808020A4F848003EE084F85E
:10A78000318087F800A0228ABA81C4F8A450796089
:10A79000E168B96032E06069B860208BB8813D46FD
:10A7A00084F83C60204607F06FFC40B185F81480C7
:10A7B0000421204601F064FDF0B9052115E084F87C
:10A7C00031A017E0E069B860208CB8813D4684F87C
:10A7D0003C60204607F058FC50B185F814800421F5
:10A7E000204601F04DFD38B9062184F8311001E012
:10A7F00084F831B0C4F8A490A07878B13A4604F156
:10A800005400D4F8A41072DF00287FF418AF94F835
:10A81000301094F8540073DF0028F6D1616B11B149
:10A8200094F831008847002009E784F83150F5E7B3
:10A83000F7B594B0174605003CD0287C9DF854101D
:10A840000024884252D000264FF0010E0D9615A824
:10A85000ADF834E00E90ADF83660E9880DAA4FF6F9
:10A86000FF70ACDF040026D19DF854002874687C8A
:10A87000A0B30F96109611961296E888ADF83C009A
:10A88000BDF83600ADF840000DA811900E9812905A
:10A89000A7F57F408DF83EE0FE3805D039460FA879
:10A8A000FFF7E2FC044621E0684600F09DF8002531
:10A8B0006F460FE00E2017B0F0BD00BF07EB450656
:10A8C000B08800F0C5F8022803D144B10FA9B088C0
:10A8D000AEDF6D1C0098A842F0D807E005E0B18813
:10A8E0000FA8FFF7C1FC0446F3E708242046E2E77F
:10A8F00038B50D46040018D0BDB12868206028790D
:10A900006074FF20207401208DF8020041F60F00D2
:10A91000ADF80000221D69460120A8DF002803D100
:10A9200029462046FFF7D6FB38BD0E2038BD38B586
:10A93000002924D0002822D00288502A1FD10546A1
:10A94000487C0C4600281AD0E9886289A81D9142EB
:10A9500015D14189022912D1216800290FD00C306C
:10A9600000F0CBFB08B1002000E001208DF80000D2
:10A97000A888ADF80200226869462046904738BD95
:10A9800070B5040012D001461C221448FEF76EFD7B
:10A990001248134D0560206850B17ADF002806D1B7
:10A9A0002068016829604068686005E00E2070BD7D
:10A9B0000B487BDF0028FAD108484FF6FF711438A6
:10A9C000084A20F8041B0549343901600021FFF7CB
:10A9D00005FA0028EBD0032070BD0000D01F002036
:10A9E000901B0020212002000149496800F0A2BF0D
:10A9F000EC1F002010B5044600F080F8002805D0B8
:10AA00002146BDE81040024802F067BF10BD0000BB
:10AA1000FC1F002070B515460E46044607F040FBAB
:10AA2000002809D0054800EB840080692A46314699
:10AA3000BDE8704001F062BC70BD0000EC1F00205A
:10AA400010B5002400F05AF800B10124204610BDD2
:10AA500070B50546002400F051F838B12946044885
:10AA600002F03BFF08B1022400E00124204670BD43
:10AA7000F41F002010B51821034802F009FF182820
:10AA800000D0C0B210BD0000EC1F002070B505461C
:10AA90000C46084607F004FB60B1284600F02EF88B
:10AAA00040B10548294600EB8400BDE870401830ED
:10AAB00002F013BF002070BDEC1F002070B50546EA
:10AAC00014460E46084607F0EBFA002812D0284636
:10AAD00000F014F800280DD00748294600EB860046
:10AAE00018301CB1BDE8704002F002BFBDE87040F4
:10AAF00002F0B3BE70BD0000EC1F0020142801D38B
:10AB0000002070470146014802F0E7BEF01F002018
:10AB10007CB5054608880C460930904201D90C20C6
:10AB20007CBD68466DDF0028FAD121880820685472
:10AB300020881B21401C80B2208029542088401C82
:10AB400080B220802844DDF801100160BDF80510B6
:10AB500081802088801D80B220809DF800104908E7
:10AB600000D0012129542088401C208000207CBD79
:10AB70007FB5044601208DF8060041F60A00ADF8C5
:10AB80000400454A01A90120A8DF00287ED12288BF
:10AB900004F13C0552B140482B46801C009042F61F
:10ABA0002920616800F0E2FD002873D1228952B1AA
:10ABB00039482B460A30009042F62420E16800F024
:10ABC000D5FD002866D1228A52B133482B46123077
:10ABD000009042F62520616900F0C8FD002859D197
:10ABE000228B52B12C482B461A30009042F6272077
:10ABF000E16900F0BBFD00284CD1228C52B12648FF
:10AC00002B462230009042F62620616A00F0AEFD0D
:10AC100000283FD1228D52B11F482B462A30009088
:10AC200042F62820E16A00F0A1FD002832D1216B14
:10AC300071B102A806F0ACFF17482B4632300090E5
:10AC4000082202A942F6232000F090FD002821D11D
:10AC5000606B58B110492B463A3100910279016876
:10AC600042F62A2000F082FD002813D1A16B81B1A9
:10AC700002A805F0CEFC08482B464230009007227F
:10AC800002A942F6502000F071FD00E002E0002829
:10AC900000D1002004B070BDEE1B002038B5028842
:10ACA0000446212A2ED011DC1D484FF003011D4D12
:10ACB0000088102A01EB004010D0112A05D11AA1FA
:10ACC00003F0EEFD4FF6FF70288038BD3B2A23D0FD
:10ACD000562AFAD18088132176DF0DE016A103F001
:10ACE000DFFD072000F06CFB08B1FFF76BF8A188CF
:10ACF0002980144802F026FF0028E6D0BDE838403D
:10AD0000FFF760B800200090A08869468FDF002818
:10AD1000DBD0FFF757F838BD8088132176DFEBE7EB
:10AD20009C1D0020481B0020446973636F6E6E6594
:10AD3000637465642E000000436F6E6E6563746516
:10AD4000642E0000E41E002010B51A4C01886068D3
:10AD500010290ED011292BD1401E606028D1FEF79A
:10AD600001FF002824D02168002921D0BDE810402F
:10AD70000847D0B900210122084600F0FFFA08B1C7
:10AD800007280FD107220221012000F0F7FA08B1AD
:10AD9000072807D104220221002000F0EFFA20B199
:10ADA000072802D0216801B188476068401C6060B4
:10ADB00010BD0000881B00202DE9F04701883B4EA4
:10ADC00040F2F3194FF6FF7510291BD011293ED020
:10ADD000122954D0502946D1C188F289841D91424C
:10ADE00041D1618902293ED18688304601F0F6FFC3
:10ADF000050038D004F10C0000F07FF9A8B3294613
:10AE000030464EE0C17B8788044601292BD1A846F5
:10AE1000284601F0E3FF050017D02F80002028729C
:10AE2000234843464A460168C5F80A104068C5F8F9
:10AE30000E0004F1100105F10A0002F09BF868729F
:10AE4000F08900280FD129462AE0042013E08088E9
:10AE500001F0C4FF040006D06068FFF73FF808B1B6
:10AE600006F072F92580BDE8F087FFE76868FFF714
:10AE700035F80028F7D0BDE8F04706F065B98788B7
:10AE80000646384601F0AAFF0400ECD02B464A469D
:10AE900006F1080104F10A0002F06CF86072214624
:10AEA0003846BDE8F04700F0ABBD0000D01F0020E1
:10AEB000901B00202DE9F04F0746858802883D4809
:10AEC000012197B08346102A09D0112A49D01A2AA5
:10AED0006CD1387AB1EB101F45D2012244E0354CD9
:10AEE000083CA068C0430B9061680BA802F019FDF4
:10AEF0000B990CA800F01EFD2C220CA96846FEF749
:10AF0000B5FA0026E946A04610E000BF09EB46006E
:10AF10005FF00004B0F804A008EB84005146001D67
:10AF200002F09BFC641C1D2CF6D3761C0098B042EA
:10AF3000ECD8142D05D317B00420BDE8F04FFEF770
:10AF400041BF2946584602F0D3FC294608F10400C7
:10AF500002F0CEFCF87B012828D016482946001DB7
:10AF600015E029461AE000220221B1EB101F01D2A0
:10AF7000012600E000260F49083901F11000041DE8
:10AF8000294682B102F0B4FC36B12946204617B0FA
:10AF9000BDE8F04F02F0ACBC2946204617B0BDE832
:10AFA000F04F02F05ABC02F058FCF5E717B0BDE8CC
:10AFB000F08F0000F41F002010B504460748007809
:10AFC00000280AD0204601F037FD204606F03EFB5F
:10AFD0002046BDE8104001F0D1BA10BDC01B0020D2
:10AFE00038B50D4604001FD0F5B1286820604FF633
:10AFF000FF70E0826889208301208DF8020041F60D
:10B000001400ADF80000221D69460120A8DF0028C9
:10B0100009D12946204605F02DFE002803D12946F6
:10B02000204605F09DFD38BD0E2038BD30B58BB0F3
:10B03000040029D041B3E08AA0F57F42FF3A25D031
:10B0400005AA204605F077FE0546ADF80000002071
:10B050000190029003900490E188ADF80410012162
:10B06000ADF808008DF8061005A8CDF80CD00490B6
:10B07000E08A01A9AEDF002804D1BDF80010A94282
:10B0800000D00C200BB030BD0E20FBE70820F9E704
:10B0900038B500291FD000281DD00288102A15D0ED
:10B0A000112A15D0502A16D130F8062F4B899A4212
:10B0B00011D10C46418902290DD1216800290AD0FD
:10B0C0000C3000F01AF838B1002006E0808801E06A
:10B0D0004FF6FF70C88238BD01208DF8000022684D
:10B0E00069462046904738BD70B504460D4608466F
:10B0F000FEF7E0F92080656070BD007800F0010087
:10B1000070470A7802704978417002207047000049
:10B110000149085C70470000082602000649095CE6
:10B120004FF0A040D0F81005C84010F0010000D04A
:10B13000012080F001007047082602002DE9FC4143
:10B140000646C0074FF000050ED0104F0024012224
:10B15000385D009500231146019503F02FF9641C1A
:10B16000042CF4D300F046F8B0070DD5074E0024A8
:10B17000361D0022305D032300951146019503F032
:10B180001DF9641C042CF4D3BDE8FC8104260200E4
:10B1900007490B5C4FF0A041D1F8042501209840ED
:10B1A00020EA0203C1F808351040C1F80C057047C9
:10B1B000042602000249085C012103F062B9000084
:10B1C000042602000249085C002103F05AB900007D
:10B1D000042602000649095C4FF0A040D0F804059F
:10B1E000C84010F0010000D0012080F0010070473D
:10B1F0000426020010B500242046FFF7DBFF641C84
:10B20000042CF9D310BD10B500242046FFF7DAFF57
:10B21000641C042CF9D310BD10B50246064B4FF048
:10B22000FF3000215C5C944201D1084610BD491CEE
:10B230000429F7D310BD00000826020070B50C4E9B
:10B240000C004FF0000530600BD0012000F06AF8D0
:10B2500008B1022004E0002000F064F800B10B20E7
:10B260002070706810B9FEF77DFC0546284670BD59
:10B27000881B002010B5002000F0D4F908B1062882
:10B2800006D1012000F0CEF908B1062800D1002037
:10B2900010BD00002DE9F0470D468146FFF7BCFFC9
:10B2A0000446042836D2DFF874801B481C4EA8F1EF
:10B2B0000C0725B3012D0ED0022D2BD104EB440039
:10B2C00030444578002D25D0B968002922D0284681
:10B2D000BDE8F047084704EB4401755C0E44717803
:10B2E00049B10E4A4FF40041093A8068FEF7B2FDB9
:10B2F00008B987F80390B17808F80410E2E780688D
:10B30000FEF7ECFD04EB4401314418F804008D789D
:10B31000A842D7D0BDE8F0870C260200841B00208D
:10B32000701F0020042801D2FFF7F8BE00207047EC
:10B330000146104810B50088042907D007290ED00F
:10B340000A2915D1BDE8104006F06CB9132176DF4B
:10B350000CE000280CD0BDE81040FEF733BDA0F58E
:10B360007F41FF3904D10448FFF73DF90828F0D1A7
:10B3700010BD0000481B00202C1E002070B50023CB
:10B38000042810D20D4D00EB4004012A02D10129FE
:10B390000CD00022094E00EB4000304461B101297D
:10B3A00006D0022906D00723184670BD0E30C2B25F
:10B3B0002A55F9E74270F7E78270F5E7701F002021
:10B3C000044A014600201279D20702D0084600F054
:10B3D0004DB87047781B002070B506461E48002403
:10B3E000C0E90161B00720D5002501221146284699
:10B3F000FFF7C4FF6D1C0446042D02D2002CF4D0CC
:10B4000013E094B940F2666204211448FEF760FC30
:10B4100004000AD1FEF74AFC040006D10F48104A86
:10B420000021001FFEF7DAFC0446F00712D00120CD
:10B43000FFF784FE74B909480A4A00210C38FEF768
:10B44000CDFC040006D10548074A01210838FEF763
:10B45000C5FC0446204670BD781B0020182602005B
:10B46000F1B6010009D001009B9C01002DE9F05FBD
:10B470006A4C054600266078B34618B184F801B0DE
:10B4800001F0AAFD664F4FF47A694FF4C87A4FF085
:10B490000108182D62D2DFE805F0AC0C0C31404DEC
:10B4A00062676B746B74BE7D7D7D7D7DACAFB2B524
:10B4B000BEBE0020FFF78EFE00284FF0000008D02F
:10B4C000FFF778FE022D02D14FF4E16008E0484614
:10B4D00006E0FFF777FE022D01D1C82000E05046BC
:10B4E000410CC0034FF4FA72801841F1000125703D
:10B4F00052000023FDF776FF01462AE00020FFF707
:10B5000069FE00284FF0000004D0FFF753FE4FF40F
:10B510004870E5E7FFF756FEDFE70020FFF75AFE29
:10B5200000284FF0000002D0FFF744FECFE7FFF7FE
:10B5300049FED4E70020FFF74DFE00284FF0000041
:10B5400002D0FFF737FE01E0FFF73CFE257041F621
:10B550009A1100223868FEF77DFC064646E000207E
:10B56000FFF716FE257008E0002051E025703DE051
:10B5700084F801800120FFF70BFE002240F6CD4148
:10B58000E8E784F801800120FFF702FE00224FF473
:10B590008041DFE77868FEF7A1FC0646D5F111008F
:10B5A00000D02EB10220FFF705FE84F802B01DE0A6
:10B5B000012816D980B2C8214843C117C90341EAFE
:10B5C0005041C0034FF4FA72801841F1000152005B
:10B5D0000023FDF707FF014600227868FEF73AFCDA
:10B5E00006460220FFF7EEFD84F802803046BDE8F3
:10B5F000F09F01F0F1FCB9E701F0EEFCB4E701F0D7
:10B60000EBFC04E001F0E8FC0020FFF7DBFD01208B
:10B61000FFF7D8FDAAE7FFF7F6FDA7E7781B0020A4
:10B620000C260200012106F0D2BD00002DE9F843EE
:10B630000546861C00208DF8000090460F464FF00E
:10B6400001096846FEF75AFC1B4C20683860D4E9B3
:10B650000001401AA16804F21C47081A0EE00121FB
:10B66000384602F058F901F06BFE0146384602F008
:10B6700052F9D4E90001401AA168081A401C864218
:10B68000EDD8B8F1000F03D0052065F3891002E072
:10B69000062065F39F50A2682168114004EB8101E8
:10B6A000C8602068304420609DF80000FEF74AFC26
:10B6B0004846BDE8F88300001827002030B48268AF
:10B6C0000468531C8360A154D0E901128A4202D35A
:10B6D00030BC02F020BB30BC70470000034803C8F8
:10B6E000814201D1012070470020704718270020B7
:10B6F00000780221FFF7CEBD05494FF0FF32082840
:10B7000041F8202002D3084480F848207047000008
:10B71000D4220020F0B54FF0FF3512B100230826E7
:10B7200001E008230C260C4C05E000BF54F8237000
:10B730007F1C04D05B1CB342F8D32846F0BD26180A
:10B740005DB286F8305044F82310002AF5D1E11894
:10B7500081F84800F1E70000D422002002490844A3
:10B7600090F9300070470000D42200202DE9F0430A
:10B770008FB01E46DDF8589015460F00804602D166
:10B780000020FEF71FFB15B90020FEF71BFB1C2154
:10B790006846FDF784FE00249DF80000039440F005
:10B7A00002008DF80000012001948DF83600049409
:10B7B00005940694ADF834800C9430788DF8300000
:10B7C00070788DF831009DF83200142120F00600C9
:10B7D000801C20F019008DF8320007A8FDF75FFEED
:10B7E0000DA807900CA808900748ADF82450ADF8B4
:10B7F0002640ADF828500B974B4607AA69460088AB
:10B80000AADF0FB0BDE8F083EE1B002070B5044640
:10B810004FF6FF750A462846AC4208D14FF48074B3
:10B820002146104604F070FDA04209D070BDFF2CE7
:10B83000FCD82146104604F05AFD08B1204670BDE0
:10B84000284670BD70B5084C050009D01034216839
:10B85000002907D008682060496828468847F6E72D
:10B860000834F4E770BD0000C0220020054A012121
:10B8700020B1012805D19170FFF7E4BF517000207D
:10B88000FAE77047C02200202DE9F05F26484168A2
:10B89000F1B3DFF898B00E688146DBF800408768A6
:10B8A0008078E11B21F07F45ED1CB0B9DFF8808086
:10B8B0004FF48030C8F84403C8F804031120FDF7A2
:10B8C0000DFF1120FDF715FF4FF0010AC8F800A089
:10B8D0002F2003F025FC89F802A0B54200D235469E
:10B8E000124BE8193C3320F07F401860DBF8001061
:10B8F0005A46091B21F07F41001B20F07F40C91CE4
:10B9000081420FD9106818602F2003F009FC00E075
:10B9100004E0BDE8F05F1120FDF7F6BEBDE8F05F82
:10B9200005F038BABDE8F09F681C002004150140FE
:10B930000010014073B58CB00646002000900D98B1
:10B9400080B100246D4621460DA801F0C6FF30B13C
:10B95000009805EB400084800098401C0090641C17
:10B96000142CF0D32C2269463046FDF77FFD0EB033
:10B9700070BD2DE9F04117880646B81D14460D46E6
:10B98000984202D90C20BDE8F081318807220629AF
:10B990000AD34FF4486C4FF6FF73614501D99942C1
:10B9A00002D17088062801D21046ECE7604501D923
:10B9B0009842F9D1994203D0984201D08142F3D8FC
:10B9C0000520E85520881221401C80B2208029548F
:10B9D0002088401C80B220804119308806F0A6FAE9
:10B9E0002188084480B220804119708806F09EFAB0
:10B9F0002188084420800020C5E7FEF7E3B9000055
:10BA000038B54A7A0F4B62B100220A72596900298F
:10BA100006D001228DF80020ADF802006846884764
:10BA200038BD0A7A62B19B684C68024619462046C6
:10BA3000FEF710FA0028F3D0BDE8384005F084BBCB
:10BA40005B68F1E7D01F0020F0B585B016460F46C1
:10BA500004461D4614220B496846FDF707FD0A48B7
:10BA60008DF80870ADF80240ADF80A608DF80C5002
:10BA7000017800222046FFF721F8684600F0FAF925
:10BA800005B0F0BD1C270200D01B002030B50446D5
:10BA900085B000211B4804F02AFC00282FD0002587
:10BAA000204600F0F8FE68B1112812D086281BD07D
:10BAB000A0F54051023903D00146204605F04CFB69
:10BAC000294607E005B029462046BDE8304001F090
:10BAD00015BC0121204601F011FC05B00021BDE894
:10BAE0003040084804F037BC142207496846FDF787
:10BAF000BDFCADF80240684600F098F9E0E705B0FB
:10BB000030BD0000991B00204C2602007FB50C467A
:10BB100010B1012004B070BD2079002638B141F683
:10BB20001D5501281BD0022826D00F20F2E7022045
:10BB3000207102960396E0680190694601A804F01E
:10BB40006BFF50B102988188E18000882081BDF8A8
:10BB50000010029804F0DEFFDCE70A20DAE70A4B67
:10BB60006A460021A01D04F013FF38B106491839B8
:10BB70008E61CE610A28CDD12846CBE70248818864
:10BB8000019804F0C7FFF5E7A81C00202DE9F04755
:10BB90000025DFF88C803CE06068002100EBC506E2
:10BBA000012032789146FDF74EFCD4E9062300EAE5
:10BBB000020701EA030C57EA0C0728D082438B43A3
:10BBC0004846C4E9062303F06DFB3278824691466D
:10BBD00001200021FDF737FCD4E9042300EA020428
:10BBE00001EA03074A4650460021FDF72CFC444079
:10BBF0004F403C430BD17078012801D0012100E077
:10BC00000021726881EA0A010AB1484690476D1C1A
:10BC1000EDB298F8000044468542BDD3BDE8F087F8
:10BC2000481C002010B50021024801F08FFE80F36F
:10BC3000100010BD342B00200E4910B50A784C7846
:10BC40000023A24212D0521CD2B20A70022A00D1A2
:10BC50000B70084A0B780C3252F823200260886877
:10BC6000104420F07F408860012010BD0360002058
:10BC700010BD0000681C002013460A460021FFF793
:10BC8000E3BE00002DE9F843104D0F4680461E46E6
:10BC900091466946286801F0B4FD040014D01C21C7
:10BCA000FDF7FDFB01202071C4F81490380BC4F897
:10BCB0000080C4E902606946286801F0C3FD04F011
:10BCC000FBFD0020BDE8F8830420FBE7E827020025
:10BCD00010B503780022072B06D2DFE803F0050435
:10BCE0000610202930000A7010BD01230B70038953
:10BCF0008B818388CB81C06888600A7410BD022262
:10BD00000A7002898A818288CA81C2688A60807DBD
:10BD1000062802D00020087410BD0120FBE7032292
:10BD20000A70C2888A810289CA81C068886010BD91
:10BD300004230B70C0888881CA818A6010BD0520E9
:10BD4000087010BD70B5064D0646002455F8241045
:10BD500009B130468847641C042CF7D370BD00003D
:10BD60009824002030B50446006887B00D468068EE
:10BD700000281FD018216846FDF791FB0195A068A7
:10BD80000590207910B1012810D107E001208DF82D
:10BD9000000020690290E068039005E002208DF821
:10BDA0000000E068000302906069049020688168E8
:10BDB0006846884707B030BD70B586B015460C00A0
:10BDC000064619D0112C17D0082C15D0142168461E
:10BDD000FDF765FBADF80260304600F053FFADF8AB
:10BDE00004000D2C0AD0862C1CD007208DF80000F2
:10BDF0000294684600F04CF806B070BD03208DF840
:10BE0000000025B12878C00701D0012000E0022001
:10BE10008DF8080000208DF80C0041F20110ADF8FB
:10BE20000A00E6E706208DF80000E2E710B50446B8
:10BE3000408800F027FFA080024801682046BDE846
:10BE400010400847A01B00202DE9F04107460024C0
:10BE5000064E074D05E000BF56F8241038468847C7
:10BE6000641CE8788442F7DBBDE8F081742200208E
:10BE7000C01B002010B50446408800F003FFA080DE
:10BE8000024801682046BDE810400847F02602003D
:10BE900001490968084700004427020070B586B0D0
:10BEA000044614216846FDF7FAFAA0890125A0F599
:10BEB0004040ADF8040020782A4E062833D2DFE84F
:10BEC00000F0320303032C48A08900F0BDF930B91B
:10BED000E08943F6FE71A0F54040884223D8A07B5C
:10BEE0008DF80800207803280FD000208DF8090075
:10BEF000A0680390606850B109208DF80000606868
:10BF00000490684603F05AFE0DE00120EEE7082099
:10BF10008DF800008DF81050F3E7A08900F094F937
:10BF200008B1E08930B17078002801D003F076FFC5
:10BF300006B070BD606820B10B208DF800007570F0
:10BF4000DFE70A208DF80000BDF8040003F0F0FFE1
:10BF5000F5E713208DF800004FF6FF70ADF80400F0
:10BF6000CFE70000B01B002038B504460E4800782B
:10BF7000A8B1A4F57F40FF380FD0684604F0CEFB8F
:10BF800078B10521017001210171C480684604F077
:10BF9000D3FB04F083FC002038BD042038BD022010
:10BFA00038BD082038BD0000B01C00200C4808B582
:10BFB000007888B1684604F0B1FB78B106210170C1
:10BFC000684604F0B9FB0748017809B10121017303
:10BFD00004F064FC002008BD022008BD082008BD54
:10BFE000B01C00205C250020F0B587B01421684605
:10BFF000FDF755FA2B4C207818B16846FFF7A2FEE2
:10C000004EE0201D01F084FCB8BB4FF010204169C8
:10C01000000400694A1C02D100EB400001012248E3
:10C0200000220161A1F54051C160204902F002F8EF
:10C03000002820D11F481C238C221D49006801F0D4
:10C04000CDFB03F0ABFB050014D0022D12D000276E
:10C050000126062D12D005A804F060FB88B10670F9
:10C060000C2D18D2DFE805F0170F170F171617164B
:10C07000171113110B2007B0F0BD11E02670676097
:10C08000BBE70820F7E7077105E0032100E0022184
:10C09000017100E0067105A804F04EFB04F0FEFB00
:10C0A0000020E8E7B01C0020581D0020F8270200FF
:10C0B000A82400206027020038B5040014D0694687
:10C0C00004F0AAFCA0B1BDF8000000EB8001094813
:10C0D00000EB8100C16849B1A17A39B1C168491E3C
:10C0E000C1600020A07238BD052038BD062038BDD3
:10C0F0000A2038BD342500201FB501A9684604F088
:10C1000047FC04B010BD07B513460A466946002037
:10C1100004F03EFC0EBD07B513460A4600216846F2
:10C1200004F036FC0EBD20B119B100680860002093
:10C130007047052070470000F8B50D46040018D080
:10C14000BDB1694604F068FCA8B1BDF800000B4918
:10C1500000EB800001EB800001210C30666801F0EB
:10C16000DAFB2E6060680C3068600120A07200204D
:10C17000F8BD0520F8BD0A20F8BD000034250020D8
:10C1800018B10323002206F011B9052070470223DD
:10C19000002206F00BB912B1022306F007B9052000
:10C1A00070470000084910B50A69042A0AD0074AF6
:10C1B000096942F8210004480121103001F0ABFB6D
:10C1C000002010BD0C2010BD901C002098240020E1
:10C1D00038B5044609480D46007858B164B169463F
:10C1E000284606F0DDF9002803D1BDF800102180B3
:10C1F000658038BD022038BD052038BDB01C002048
:10C2000010B504460E48007898B1A4B121880229DF
:10C2100013D80C4A01EB810002EB8002608852893E
:10C22000C31C934209D806F0AFF90020208060803B
:10C2300010BD022010BD052010BD042010BD00005F
:10C24000B01C00203425002043F6FE71A0F54040CC
:10C25000884201D8012070470020704710B504467D
:10C260000078182802D1FEF705FC207010BD10B52B
:10C2700004460078182802D1FEF7FCFB207010BDA0
:10C2800070B50D460446B0F89810D0F8940001221D
:10C29000FEF7B0F800B1057004F13C0204F194011E
:10C2A00004F1540072DF70BD70B5134600220646DB
:10C2B0001546862902D0112902D002E0012200E0B1
:10C2C00001250D4C73B1A179FEF7F8FB2A4661797F
:10C2D0003046FEF7F3FB0022A1783046FEF7EEFB76
:10C2E000002203E0A178FEF7E9FB2A466178304698
:10C2F000BDE87040FEF7E2BBD81B0020F7B517463B
:10C300000E0011D00098002560B100242146684637
:10C3100001F0E3FA18B1A0B23946B0476D1C641CB5
:10C32000142CF3D32846FEBD0020FEBD406804F067
:10C3300015BA00000EB516A19DF8080020F00F00F8
:10C34000401C20F0F00010308DF808000A2202A8EE
:10C350007CDF08B1FDF736FD4FF4886078DF08B167
:10C36000FDF730FD00204FF4C87100900190ADF84A
:10C370000400ADF800104A00ADF80220ADF8061038
:10C3800068467ADF002801D0FDF71CFD0EBD0000D5
:10C390004E6F726469635F525343000070B508B119
:10C3A000012070BD194C0025207B08B1257301E0E8
:10C3B00000F0A0F82078082826D2DFE800F0250455
:10C3C000080C10251420BDE8704000F021B8BDE82D
:10C3D000704000F07DB8BDE8704000F05FB8BDE887
:10C3E000704000F03BB86088084900EB80002839B5
:10C3F00001EB80004068BDE8704003F0AFB96560B4
:10C40000BDE8704003F0B8B90F2070BD5C25002076
:10C410001149F0B48A1C00200346A1F128050C182C
:10C42000A67A4EB1A37200EB800405EB8404E668A3
:10C4300016B9247C012C0AD0401C80B20228EED30D
:10C440000B704B804B60F0BC41F61D507047108064
:10C45000F0BC00F03DB800005C2500200C4841888D
:10C4600001EB8102A0F1280101EB8201CA6852B1FF
:10C470000521017007480221818001680023012203
:10C48000054801F041BD042202704968F6E700004A
:10C490005C250020B81C0020581D002038B50A4932
:10C4A000084803240B684268898803EB810153889C
:10C4B0000470DB1C00201B0400909B0B034801F060
:10C4C00093FE38BD5C250020B81C0020581D0020BC
:10C4D000074910B54888091D04F0EEFA18B1BDE807
:10C4E0001040FFF7DBBFBDE81040FFF7B7BF00000B
:10C4F0005C250020F0B51F481F490125067802245D
:10C500008B88A0F12802082E19D2DFE806F0041863
:10C51000181B222F2F170189491C018100214180FE
:10C5200080F80C1001EB810312F8233043B1002393
:10C530004418491C89B2A3720229F3D30570F0BDD7
:10C540000123F5E742685288D21C1A448A8004709D
:10C55000F0BD46880D6806EB860602EB860256683B
:10C560000E60556013818C80062100E00721017068
:10C57000F0BD00005C250020B81C002030B501880B
:10C580008488224D85B0502924D0522902D05429C4
:10C5900031D103E0204600F07DFE2CE014221C493E
:10C5A0006846FCF763FFADF80240204600F06AFBE6
:10C5B000ADF8040000F022F9002269792046FEF768
:10C5C0007DFA002229792046FEF778FA6846FFF7BF
:10C5D0002DFC10E0017B01290DD1817A01290AD1BE
:10C5E0000089A0F52451023905D10121204600F02F
:10C5F00085FE05F00BFD00220649E878FEF70AFAF1
:10C6000005B0BDE8304004F059BE0000981B002082
:10C610007426020001A0010010B50446007800282D
:10C620000FD1608800F036FE608800F081F90028A4
:10C6300007D00449608801220979BDE81040FEF75F
:10C640003DBA10BD981B002010B5124C0020207080
:10C65000FEF710FAA070FEF70DFAE070FEF70AFA86
:10C660002071FEF707FA6071A17818290FD0E178E0
:10C6700018290CD02179182909D0182807D00121B0
:10C68000601C03F02DFE01202070002010BD03204F
:10C6900010BD0000981B00207CB5044600780828D7
:10C6A0002FD1607A38BB207A4FF6FF7501280DD064
:10C6B000072802D0082824D11EE0A08800F020FA24
:10C6C000A8421ED0012100F019FE1AE0A0886A4697
:10C6D000012103F08BF970B90198007858B1A08856
:10C6E00000F00EFAA8420CD0084901220979FEF7A1
:10C6F000E5F904F0E3FD04E004480021401C03F0E8
:10C700002AFEBDE87C4005F081BC0000981B00209B
:10C7100010B504460A4841782046FEF7B7F968B1DB
:10C720000848002101EB410200EB82025288A2423C
:10C7300001D1C8B210BD491C1429F3D3FF2010BD8C
:10C74000AA1B00206420002070B5094D094E00246A
:10C7500004EB440005EB800071784088FEF796F901
:10C7600020B1641C142CF3D3FF2070BDE0B270BD67
:10C7700064200020AA1B00202DE9F04180460246DB
:10C7800001200021FCF75FFE1A4F05460E4678682F
:10C79000FDF7A4FB00280CD1174CD4E90621104664
:10C7A0002A4001EA06031A4305D0A843B143C4E96D
:10C7B0000601BDE8F081404602F074FD30B1D4E9D5
:10C7C000040128433143C4E9040105E0D4E904101D
:10C7D000A943B043C4E90410D4E906012843314316
:10C7E000C4E90601A1687868BDE8F0410022FDF7C0
:10C7F00031BB000050270200481C00201CB5054A30
:10C80000D2E90212CDE900120022694603F013F9C1
:10C810001CBD00008C26020003484FF6FF7181808A
:10C820000121017000207047A41B00202DE9FC416C
:10C83000804600F027FA002403250127A0F57F4158
:10C840002646FF3908D06A46082103F0CFF818B908
:10C850000198841D8688056832462B46214640464D
:10C86000B1DF042804D0082804D00B2808D002E047
:10C87000112000E00020002F00D10B20BDE8FC813A
:10C880000027A80701D50125E6E73443F5D00024A9
:10C8900026460325E0E72DE9FC41804600F0F2F949
:10C8A0000646A0F57F40FF380ED001252A466D1CB4
:10C8B0000027ADB26B460821304603F0C1F80400F2
:10C8C00006D0072C25D025E043F20200BDE8FC810C
:10C8D000019903230A1D0B604046891DB2DF040045
:10C8E00004D00C2C09D0052C09D009E032460821CF
:10C8F000104603F01BF904460CE0012700E0002479
:10C900000821304603F0FEF800B10324002FCDD1FA
:10C9100000E00C242046D9E704488088A0F57F4138
:10C92000FF3901D004F0D4BC70470000A41B0020E4
:10C930000EB502A9019100F0A5F96A46012103F0A4
:10C9400055F808B100200EBD019800780EBD00001A
:10C950002DE9F04107464FF6FF760A48B3DF10B1E4
:10C960000320BDE8F081074C43F20305A41E3246C4
:10C9700061883846AFDFA842F3D16088401C6080F0
:10C98000F5E70000A61B0020428800EB82020C3273
:10C990008A4201D9022070478188A1F57F42FF3A7F
:10C9A00003D0008808B100207047012070478842FA
:10C9B00004D20068401C01D001207047002070475D
:10C9C0003EB5027802230C46B3EB520F17D1B0F8F4
:10C9D0000110ADF80010C1788DF802108188ADF813
:10C9E000041080798DF8060002AA01A92046FDF7FF
:10C9F0002BF9032202A96846FCF763FD08B1002069
:10CA00003EBD01203EBD000010B50C46FFF780FE84
:10CA1000FF280CD0074900EB400001EB8000416883
:10CA200021600189A180807AA071002010BD0520BD
:10CA300010BD00006420002070B5018890B010295E
:10CA400059D1011D28226846FCF710FD9DF804000D
:10CA50004FF6FF76032134466D46B1EB500F2AD0D6
:10CA600003F01AF99DF8040040080ED001280CD0FC
:10CA7000022820D118E00C99281D1131FDF74DF83E
:10CA800018B100BFBDF8284015E00BAA0AA907207D
:10CA900003F0D6F80028EED10DE00C99281D491CB2
:10CAA000FFF78EFF0028EDD10BAA0AA9072003F09B
:10CAB000C7F80028F1D1BDF80000291D00F038FEAC
:10CAC000B44218D0BDF80000214600F0C5F8BDF80A
:10CAD0000000ADF82A000020ADF82C40074E8DF87C
:10CAE00028000AAD044600BF56F82410284688479F
:10CAF000641C022CF8D310B070BD0000A026020008
:10CB0000094A002101EB410332F82330834205D169
:10CB100001EB410002EB800040887047491C14295A
:10CB2000F0D34FF6FF707047642000203EB50C46EE
:10CB3000054603F0B1F80BE0BDF80000A04207D0B5
:10CB40002846029900F02EF810B1BDF800003EBD55
:10CB500001AA6946072003F073F80028ECD14FF6CC
:10CB6000FF703EBD10B50D4C18200D4A60700020BE
:10CB70004FF6FF7100EB400302EB8303401C59802A
:10CB80001428F7D3FDF776FF6070182803D0012032
:10CB90002070002010BD032010BD0000AA1B002043
:10CBA000642000202DE9F0410C46054600F11107F4
:10CBB00001F111061022491C401CFCF782FC48B907
:10CBC000681C00F0F9F928B1601C00F0F5F908B113
:10CBD000012400E0002431463846FCF79EFF3B78F4
:10CBE0000222B2EB530F0CD00321B1EB530F08D04C
:10CBF0003378B2EB530F04D0B1EB530F01D00121C6
:10CC000000E00021084201D18C4302D00120BDE8A0
:10CC1000F0810020FBE7018811B9421892780AB12F
:10CC200001207047491C0829F7D30020704710B530
:10CC30000C460346FFF7EFFF00280AD0188821882A
:10CC4000884205D10822A11C981CFCF73AFC08B1C7
:10CC5000002010BD012010BD03F0BEB970B5044620
:10CC6000FFF74EFF0546204602F0C3FE4FF6FF7168
:10CC700004468D4203D014B9284603F0ADF920468E
:10CC800070BD000010B5FFF743FDFF2805D0044933
:10CC900000EB400031F8200010BD4FF6FF7010BDD2
:10CCA000642000203EB5044602F0F6FF0EE0019934
:10CCB00020464631FFF7BBFF28B9019920462A31AB
:10CCC000FFF7B5FF10B1BDF808003EBD6A4602A9E6
:10CCD000072002F0B5FF0028E9D14FF6FF703EBDF6
:10CCE00010B50A4941600A4800F012FE58B902F036
:10CCF00057F907491C238C22087404488C39001FFB
:10CD0000006800F06BFD002010BD0000EC27020061
:10CD1000F82500202DE9F0412D4F002518B17D6048
:10CD20000120BDE8F0810879012258B1294E01287F
:10CD30000CD0274C4FF002080834022821D00328D9
:10CD400042D128E00A7102F017FD3BE05FF00000DD
:10CD500000EB800116F82110022908D0401C80B297
:10CD60000228F5D33A707D6041F61D50D9E700EBFB
:10CD7000800006F8205006EB8000406802F0EEFCD0
:10CD800020E00D71A4F804800023012212482168DC
:10CD900001F0BAF816E00D71206802F0DFFC0D49D1
:10CDA00023682831498801EB810206EB8201D1F822
:10CDB00004C0C4F800C04B60A3880B81A4F80480B1
:10CDC00006F822500028ACD07D600E20A9E70000B4
:10CDD000B01C002034250020581D002001460348C7
:10CDE00002888A4200D0002070470000BC1F00204B
:10CDF0002DE9FC5F0E008346DDE90C47C6F100001B
:10CE000098469246814600D40846012503E000BFBB
:10CE100090FBFAF06D1C5045FADAA84500D945465A
:10CE200024B1002E01DB780700D5641EB80702D5B7
:10CE3000B8F1000F0AD0F80708D13CB1A54205D2DD
:10CE400020215846641EFEF739FCF6E7002E02DA70
:10CE50004E462D2102E0780703D52B215846FEF7D8
:10CE60002DFC07F0030002280BD1B8F1000F08D108
:10CE70003CB1A54205D230215846641EFEF71EFC87
:10CE8000F6E7CDE90047434652463146584605F09D
:10CE900063F8BDE8FC9F000070B50D4604460068CD
:10CEA0004FF4887102F001F94FF49071206802F09C
:10CEB000FCF84FF49271206802F0F7F84FF4A27179
:10CEC000206802F0F2F820681249C0F804132068C4
:10CED0006907000B40B2090E002806DA00F00F00C7
:10CEE00000F1E02080F8141D03E000F1E02080F85C
:10CEF000001420680121000B40B200F01F02914095
:10CF00004009800000F1E020C0F88012C0F8001154
:10CF100070BD000010030200024600201268930753
:10CF200002D0530702D47047500714D502F0030013
:10CF3000012802D002280CD105E0C2F383100B684F
:10CF4000801C184404E00223086803EB925210444A
:10CF5000086001207047086800EB9253C2F3891003
:10CF6000401CEEE70248007A002800D001207047FC
:10CF7000F8250020F0B58488A518944200D82246F0
:10CF8000A41AC288D6189A4200D81346D21A4B88DF
:10CF90000788BB420CD34088834209D88888A042C6
:10CFA00006D3A84204D8C888904201D3B04201D920
:10CFB0000020F0BD0120F0BD0021425C0AB101203B
:10CFC0007047491C1029F8D300207047800701D012
:10CFD00000207047012070470A4810B5807860B182
:10CFE000002401E0022C06D02046FEF7E3F8641C82
:10CFF000042CF7D310BD0324F6E7BDE81040FEF77C
:10D00000F9B80000781B002003480179C90702D055
:10D010000078FEF72BBA7047781B0020172101809B
:10D020004180002101714171704700002DE9FE4FE0
:10D030002B4D984691460F00824601D000260DE008
:10D04000684600F0A1FB6A460021504602F03DFC14
:10D050002878009E10B99DF8090098B14A463146DB
:10D06000504604F04FFC0446014600225046FFF7AC
:10D070001BF90D2C32D008DC84B3082C2ED00B2CDD
:10D080000BD12BE00520BDE8FE8F112C10D0862C93
:10D090001AD0A4F54050023820D00325B8F1000F73
:10D0A00004D0324621465046FEF786FE2846EAE77F
:10D0B0003A4629795046FDF701FD4A46E97850463F
:10D0C000FDF7FCFC0025E9E73A4629795046FDF7D3
:10D0D000F5FC4A46E9785046FDF7F0FC2546DDE7C9
:10D0E000D81B00202DE9F041204F0E46154604467E
:10D0F0003978FDF7CBFC002835D0204602F0DCFB68
:10D1000050B32046FFF7BEFD80462046B978FDF7B4
:10D11000BDFC08B1012700E00227204602F074FEA2
:10D120000028404602D0FFF799FD0DE0A8F57F41A9
:10D13000FF3909D0072102F0E5FC010004D00529E0
:10D1400002D0204604F01CF82B46324639462046D1
:10D15000BDE8F041FEF778BC2A4631462046BDE8DE
:10D16000F041FEF789BDBDE8F0810000D01B002032
:10D1700070B5094D0646E978FDF788FC0446297923
:10D180003046FDF783FC014622463046BDE870403C
:10D190000123FFF74BBF0000D81B00202DE9F0470B
:10D1A000394E002780463D46DFF8E090D6F804A0CF
:10D1B00057E003D00446D0F81C8035E099F80020F1
:10D1C00002EB4201521CD2B289F8002009EBC101E6
:10D1D00099F80230091D9A4201D189F80050486837
:10D1E0000A780446012A12D0022A02D0032A3BD12F
:10D1F00008E004F04DFD00B10127257434E005740A
:10D20000C06900E070680028F9D170602CE0207CD3
:10D2100050BB88686060C868A0600869E0604869C1
:10D22000A061F07800B165606268B168184B501A6F
:10D2300020F07F40984202D2A168084406E0881A94
:10D24000A16820F07F40814202D9081A206000E0E6
:10D25000256065600120A56020742046E56104F02A
:10D26000F9FCB8F10000A4D199F8001099F8010078
:10D270008142A3D117B97168514502D00120BDE8A0
:10D28000F0870020FBE70000681C002074230020CA
:10D29000FFFF7F0030B585B00546002414216846A5
:10D2A000FCF7FDF8A5F57F40ADF80250FF3815D02A
:10D2B0002846FFF7BBFA98B10B2815D0112811D0DA
:10D2C000A0F54051023903D00146284603F044FF3F
:10D2D00009482246C1782846FDF7F0FB05B030BD6D
:10D2E0000E2002E00124F3E70F208DF800006846CD
:10D2F000FEF79CFDECE70000981B00200A4602495F
:10D300008978FDF7DBBB0000981B0020F8B50546C7
:10D3100000780C46002620420FD100208DF8000036
:10D320006846FCF7EBFD2878204202D120432870A4
:10D3300001269DF80000FCF705FE3046F8BD000010
:10D340002DE9FF410026234800F0DFFA2148001FA5
:10D35000074600F0DAFA204C60680090A56800E00B
:10D3600000986946284004EB80000C30FFF7D4FD9C
:10D370000028F5D101AA009901EA050304EB830313
:10D38000491CDB6842F82030401C00910228F2D38F
:10D39000019800F0030001280BD0022810D1019859
:10D3A000032101EB90500099BDF80A6001EB900059
:10D3B00005E00198BDF80A60C0F3831008440090AE
:10D3C000384600F09FFA08B10098606004B030461B
:10D3D000BDE8F081302B0020182700204FF40046D4
:10D3E00088B03146002001F0CDFA08B1FCF7EAFC24
:10D3F00001F038F9FCF704FD08B1FCF7E3FC4E4AF4
:10D4000001214E48FCF7EAFC08B1FCF7DBFC4B4875
:10D410004B4A0121001DFCF7E1FC08B1FCF7D2FCEE
:10D4200048490320FDF7D8FF08B1FCF7CBFC69465B
:10D430000020FDF703FF08B1FCF7C4FC9DF80000D5
:10D44000022877D05FF0000401F0BAFB08B1FCF7C6
:10D45000B9FC01F04BFD08B1FCF7B4FC00276946AC
:10D460000120009701F0D6FB08B1FCF7ABFC684641
:10D4700001F04EFC08B1FCF7A5FCFEF75BFF0021B4
:10D48000314800F0D8FA08B1FCF79CFCFCF786FBA9
:10D4900003F0CAFF03F088FE1C216846FBF7FFFF7C
:10D4A0004FF42030CDE900704FF4702002902648F0
:10D4B00003251C388DF80C504089ADF80E00234828
:10D4C0000590234806908DF810706846FDF758FACD
:10D4D00008B1FCF777FC02F0DDFE08B1FCF772FC46
:10D4E0001C4803F07BF808B1FCF76CFC1A481BA140
:10D4F000008805EB004001F0D3F9104D00224FF4F5
:10D5000080312868FCF7A6FC08B1FCF75BFC3146CB
:10D5100000226868FCF79EFC08B1FCF753FC20462B
:10D52000FCF770FB01F0ACF80028FBD101F05CFBCC
:10D53000F8E7FFE7012487E725A20100FC250200A8
:10D54000F50B020031B301001C1E002069F501003B
:10D55000FBB90100490102009C1D002052756E6E4E
:10D56000696E6720537065656420616E6420436155
:10D5700064656E6365206578616D706C6520737499
:10D5800061727465642E000070B5144682880E4680
:10D5900005462088111D0144921C994201D8FE2A9B
:10D5A00001D90C2070BD521C32542088FF21401C30
:10D5B00080B2208031542088401C80B220808119A4
:10D5C000288804F0B3FC2188084480B22080AA880F
:10D5D00042B1A96841B13044FBF748FF2088A988CF
:10D5E00008442080002070BD072070BD2DE9F04761
:10D5F000C7880446181D16468946B0FBF7F1B0FBF4
:10D60000F7F207FB12009A193A44D21CB2FBF7F268
:10D61000DDF820A001E02468491E0029FBD13D1A55
:10D620008846B54216D818E0BAF1000F05D0211887
:10D6300009EB08002A46091D04E0204409EB080113
:10D640002A46001DFBF712FF00202468761BA84421
:10D65000B74201D9354600E03D46002EE4D1BDE891
:10D66000F087000030B5024659B101F0B7F900214A
:10D67000074C09E004EB810315685B88AB4202D1DB
:10D680001160002030BD491C8142F3D3052030BD1C
:10D690006C1D0020F8B50F46017814460546012997
:10D6A00001D1687830B12088821C9A422DD8012996
:10D6B00002D006E00720F8BD69780144891C994230
:10D6C00023D8181A801E86B2ADF800602188B81CD5
:10D6D000084469467DDF0028EDD12878022805D16D
:10D6E000BDF80010B14201D809210AE00821012843
:10D6F00005D16878B04202D8ADF8000001E0ADF87D
:10D700000060BDF80000FE2801D90C20F8BD228879
:10D71000401CB8542088401C80B220803954208896
:10D72000401C2080BDF80010084420800020F8BD77
:10D7300070B505460C004FF0FF0020D04FF6FF7685
:10D74000B5421CD00E48012241782846FDF7B6F9B3
:10D750002846FEF7DDFFFF2803D1FEF7F5FFFF287F
:10D760000DD0084B00EB400203EB82014D8023F803
:10D77000226022684A60A2880A81A2798A7270BDFA
:10D78000AA1B002064200020034A00219268C0E9FF
:10D790000021816070470000D81B002070B54FF653
:10D7A000FF750E46A84201D1002000E0401C84B263
:10D7B00008E02146304602F0C2FD08B1204670BDA7
:10D7C000641CA4B2FF2CF4D9284670BD10B5FBF739
:10D7D0006CFD08B1002010BD112010BD10B531B195
:10D7E000B2FBF3F403FB14241CB1092010BD0E207E
:10D7F00010BD01600021416081608281C3810846C3
:10D8000010BD70B50C460546FBF704FD002802D09C
:10D8100021882868084470BD10B50A8849888A4262
:10D8200003D1FBF739FD012010BD002010BD70B5FC
:10D830000C460546FBF713FD002802D061882868D6
:10D84000084470BD10B50A8849888A4203D1FBF7A5
:10D85000FDFC012010BD002010BD01F01F030122BE
:10D860009A40D243490900EB8100114600F059B8B3
:10D870000A4601F01F030121994010B552090C46D8
:10D8800000EB820000F05DF8204000D0012010BDC8
:10D890002DE9F04180460D460024481E012101EB90
:10D8A000501716E058F82400C04390FAA0F0B0FAE0
:10D8B00080F020280CD200EB4416AE4208D231464C
:10D8C0004046FFF7D5FF0028ECD13046BDE8F08197
:10D8D000641CA742E6D82846F8E74A0950F8220017
:10D8E00001F01F0201219140084000D00120704743
:10D8F00001F01F0301229A40490900EB8100114603
:10D9000000F029B8002100F017B8012100F023B879
:10D91000012100F016B808B56A46FBF712FD009821
:10D9200008BD08B56A46FBF7F2FC009808BD08B5CB
:10D930006A46FBF706FD08BD08B56A46FBF7E7FC3B
:10D9400008BD08B56A46FBF7D5FC08BD08B56A46B0
:10D95000FBF7C4FC08BD08B56A46FBF7CBFC009892
:10D9600008BD08B56A46FBF7F9FC009808BD38B554
:10D97000044600258DF800506846FCF7BFFA216880
:10D980006268086890420ED9401E08600178A38A38
:10D99000E26801FB0325227A2168101AC0B20A79D5
:10D9A000824200D208719DF80000FCF7CBFA2846AD
:10D9B00038BD38B5054600208DF800000C46684695
:10D9C000FCF79CFAE868A98A201AB0FBF1F12A68F2
:10D9D0001068431C136001709DF80000FCF7B2FA58
:10D9E00038BD10B530B1017A42680368891AC9B2EE
:10D9F0001A6006E00E2010BD03681A68541C1C60F3
:10DA00001170491EC9B2F7D20068002101710846A1
:10DA100010BDC20800F007030120895C984008404F
:10DA2000704710B5C20800F00703885C01249C40D1
:10DA30002043885410BD10B560B1C160172120F893
:10DA4000021B20F8021B1B2100F8021BFFF7E6FA5D
:10DA5000002010BD0E2010BD7CB50C468188002929
:10DA600033D102880025102A06D0112A09D03A2A7B
:10DA70000BD0552A2ED129E00146204601F082FD27
:10DA800028E0A01DFFF7CAFA24E02246408934F8B6
:10DA9000063F834200D818466080172800D217201E
:10DAA0006080D06878B1607968B1174BD3E9000322
:10DAB000CDE90003ADF802106088ADF80400D3682A
:10DAC000694610469847657125717CBD0146204620
:10DAD00001F09AFDA07A0028F7D02846E188A5DF5A
:10DAE000012670B11128F0D001F0D0FA02460748A3
:10DAF00007A1008802B006EB0040BDE8704000F0CE
:10DB0000D3BEA572E6727CBDA82602006C1D002063
:10DB100073645F626C655F67617474635F6578638B
:10DB200068616E67655F6D74755F72657175657349
:10DB30007428292072657475726E65642025732EB1
:10DB40000000000020B10278DE2A03D008207047D0
:10DB50000E20704741800020704760B159B10278B3
:10DB6000DE2A0AD009684160DE2101704FF6FF719C
:10DB70004180002070470E207047082070477FB515
:10DB8000054600294DD0002D4BD008780C46DE28E4
:10DB900047D1A8886188884202D1204604F086FADD
:10DBA0002888012825D002283BD011283AD05128B6
:10DBB00037D135F8040F6188884232D1A978A81C82
:10DBC00002292ED1017A042903D0062901D0052982
:10DBD00027D10021009102228DF8002001914FF4FD
:10DBE000C07202910391ADF80420007A05280FD08D
:10DBF00010E0297A2046012913D1A9884288914250
:10DC00000FD10121017204B0BDE8704004F04EBA9A
:10DC1000ADF8041028886946B0DF002801D061689B
:10DC200088477FBDA88861888842FAD14FF6FF7087
:10DC300060807FBD00F180400068002800D0012096
:10DC4000704708B500F18040002101600068009035
:10DC500008BD000070B50B4C207808B185250FE099
:10DC60000020A06060602061E060074801F03AFA9F
:10DC7000054601F095F908B901F01EFA012020705F
:10DC8000284670BDC02200206DB8010038B50025BF
:10DC90008DF800506846FCF731F9074CE068401EEB
:10DCA000E060E06810B901F02DFAA5709DF8000061
:10DCB000FCF748F938BD0000C022002070B50646C8
:10DCC00004780C4888B0154640F82420094A0869B1
:10DCD000121D42F8240020226846FBF7C7FB04947B
:10DCE0000DB1054A00E000226946301D01F032FB0B
:10DCF00008B070BD381C0020091E02000FB408B522
:10DD00000399002904D004AA00926A4600F00FF893
:10DD100001B05DF814FB10B582680446002A05D0F6
:10DD2000D4E90403216898470020A06010BD2DE9C4
:10DD3000FC4791460C00804676D014F8011B39B19F
:10DD400025290ED04046FDF7B9FC20780028F4D1F3
:10DD500098F80C00002867D04046BDE8FC47FFF764
:10DD6000DABF0020012221782B291BD02D2902D0D7
:10DD7000302908D102E040F0010001E040F002004B
:10DD8000641C002AEFD100252A290ED02178A1F1A8
:10DD900030020A2A11D205EB850201EB4205641C10
:10DDA000303DF1E740F00400EAE7D9F800100B1D20
:10DDB000C9F800300968641C0D44217800232E291D
:10DDC0000BD114F8011FA1F130020A2A05D203EB8E
:10DDD000830201EB4203303BF3E76C290DD0682945
:10DDE0000BD0692921D00BDC252918D0582931D036
:10DDF00063290ED0642915D117E014F8011FECE750
:10DE0000702969D0732932D075291BD0782909D19E
:10DE100020E0D9F80000011DC9F800100178404643
:10DE2000FDF74CFC641C90E76CE0D9F800100A1D6B
:10DE3000C9F800200968CDE900500A224046FEF7E3
:10DE4000D7FFEFE7D9F800100A1DC9F800200968CC
:10DE50000A2206E0D9F800100A1DC9F80020096856
:10DE60001022CDE90050404604F076F8DAE7D9F800
:10DE7000001000270A1DC9F800200E68C00705D150
:10DE800012E04046761C7F1CFDF718FC3178002913
:10DE9000F7D104E0202140466D1EFDF70FFCBD4286
:10DEA000C0D9002DF6D1BDE74EB13046FBF702FBDD
:10DEB000074604E0202140466D1EFDF7FFFBBD42F2
:10DEC00006D9002DF6D103E04046761CFDF7F6FB9F
:10DED00031780029F8D1A5E7D9F80000011DC9F86B
:10DEE0000010056830214046FDF7E8FB78214046E8
:10DEF000FDF7E4FB08200021CDE9000103461022D4
:10DF00002946B0E7BDE8FC872DE9F84F2B4E040009
:10DF10009A4630884FF001031546894603EB0040CE
:10DF200024D0216800292BD0002D32D062684946C8
:10DF30004FF010071268A2F1010C1CEA090F11D171
:10DF400098466A432046FBF701FE00282AD0206845
:10DF500053462A46066901B049462046B446BDE804
:10DF6000F04F6047164B17A2009721E00E21009159
:10DF7000134B1EA21FA100F0A6FC0E20BDE8F88FD7
:10DF8000082100910E4B26A21AA100F09CFC08204B
:10DF9000F4E7092100910A4B24A216A100F093FC9A
:10DFA0000920EBE700973188054B214A08EB014037
:10DFB00010A100F088FC1020E0E700008C1D00207C
:10DFC000D3270200616464725F69735F7061676583
:10DFD0005F616C69676E656428705F66732C207082
:10DFE0006167655F6164647229000000705F667339
:10DFF00000000000257320636865636B206661691B
:10E000006C656420696E20257328292077697468FF
:10E010002076616C756520307825782E0000000030
:10E02000705F66732D3E705F617069006C656E0095
:10E03000D02A020038B503000F484FF001054FF019
:10E040000E04008805EB004009D061B119600C682E
:10E0500001B0A446BDE83040114618466047074B62
:10E0600007A2009402E0054B07A2009408A100F06B
:10E070002AFC0E2038BD00008C1D002088270200DD
:10E08000705F667300000000705F617069000000DF
:10E09000257320636865636B206661696C65642025
:10E0A000696E202573282920776974682076616C51
:10E0B000756520307825782E000000002DE9F041AC
:10E0C00028B1016819B1C969BDE8F04108470D4D93
:10E0D0000D480024461B14270DE000BF04EB84000C
:10E0E00005EB8000016829B1C969884710B101209A
:10E0F000BDE8F081641CB6FBF7F0A042EED800202A
:10E10000F6E70000581D00206C1D00200448012186
:10E110004174007A08B10020704701207047000068
:10E12000F8250020012801D0032808D10449002245
:10E1300001284A7400D00020087402F05FBB7047C9
:10E14000F825002070B50246022801D0032A45D1E7
:10E15000234C207A002841D0012833D0022831D125
:10E1600020480023022A006802D0032A2AD11BE09B
:10E17000E360017911B1012924D10DE0D0E90565F1
:10E18000711B4FF48056B14200D33146294481615E
:10E190004569A9420ED015E00169491C0161426937
:10E1A00091420FD1237213E0E168491CE160082914
:10E1B00008D9E3602372022A0AD00D21FDF7D2FDAF
:10E1C00002F0C2FA607C28B1BDE8704000F0EEBEFB
:10E1D0000021F3E7BDE8704002F010BB70BD000005
:10E1E000F8250020D41C00202DE9F84F3A4D0400FA
:10E1F0008B4628884FF00106DDF828A09846914606
:10E200004FF00E0106EB00401AD0B9F1000F1BD001
:10E210002168002920D00921B8F1000F25D06268BB
:10E220005368B8FBF3F703FB1782002A21D02B4B6E
:10E230002BA2009135A100F046FB0920BDE8F88F24
:10E24000264B3DA2009102E0244B3DA200912FA15C
:10E2500000F039FB0E20F1E7082100911F4B3AA294
:10E260002AA100F030FB0820E8E71C4B39A20091FE
:10E27000E0E75846FBF764FC102798B14846FBF7E7
:10E280005FFCB0B1424659462046FBF75FFCB8B18F
:10E29000CDF800A0206843464A46C5685946204646
:10E2A000A847CBE7009728880C4B06EB00402AA232
:10E2B0000CE000972888094B06EB00402CA205E0F3
:10E2C00000972888054B06EB004032A20FA100F012
:10E2D000FAFA1020B2E700008C1D0020C0270200CF
:10E2E00021286C656E202520705F66732D3E705F5F
:10E2F000666C6173685F696E666F2D3E70726F67E2
:10E3000072616D5F756E697429000000257320636A
:10E310006865636B206661696C656420696E2025A1
:10E3200073282920776974682076616C75652030C0
:10E330007825782E00000000705F667300000000F2
:10E34000705F737263000000705F66732D3E705FD4
:10E35000617069006C656E00616464725F69735F0F
:10E36000616C69676E656433322864657374290073
:10E37000616464725F69735F616C69676E65643361
:10E3800032282875696E7433325F7429705F737236
:10E3900063290000616464725F69735F7769746800
:10E3A000696E5F626F756E647328705F66732C2090
:10E3B000646573742C206C656E29000070B541EAA9
:10E3C0004201DDE904564FF0A04441EA830141EAED
:10E3D000052104EB800041EA0641C0F8001770BD3A
:10E3E00070B541EA4201DDE904564FF0A04441EA2C
:10E3F000830141EA052104EB800041EA0641C0F8AF
:10E40000001770BD70B541EA4201DDE904564FF0D6
:10E41000A04441EA830141EA052104EB800041EA7E
:10E420000641C0F8001770BD1CB5002100910B46D5
:10E4300001220191FFF7E6FF1CBD1CB500220B462F
:10E44000009211460192FFF7DDFF1CBD1CB50021B3
:10E4500000910B46012201911146FFF7D3FF1CBD2D
:10E460004FF0A04202EB8000D0F8002722F44032A7
:10E47000C0F80027D0F8002742EA0141C0F8001791
:10E48000704701224FF0A043824011B1C3F8082524
:10E490007047C3F80C25704718B5084B6C4601440B
:10E4A0001B68009306E000BF54F82030D3F8103505
:10E4B000401C08C28142F7D818BD0000482702005E
:10E4C000034908B50844002101600068009008BDB8
:10E4D0000060004002494058012800D000207047E9
:10E4E0000060004030B5124B01460020D3F81044C4
:10E4F000224609E0157A854205D1401C0A28F7DB3F
:10E500004FF0FF3030BD5268002AF3D1421CF9D0E1
:10E510000872D3F810242AB152684A60D3F8102444
:10E52000516030BD0022C3F810144A6030BD0000B5
:10E5300018270020F0B595B01C4615460F46084632
:10E540001A9E00F01BFB182109A8FAF7A8FF0E96E7
:10E55000CDE909540023082203A9384600F023FB23
:10E5600005980690BDF81000ADF81C00BDF812002B
:10E57000ADF81E0000208DF821000398082600F059
:10E580000300012802D0022818D032E00398334655
:10E59000850AC0F3C2008DF8200003980FA9C0F3CC
:10E5A0008314A200384600F0FEFA09A8009006ABDA
:10E5B00022460FA9284600F03DFA1AE00398840D80
:10E5C000C0F3C2008DF82000082C01D2254600E0DF
:10E5D000082533462A460FA9384600F0E4FA2E44AF
:10E5E000641B09AB06AA29460FA800F075F9002C98
:10E5F000EAD1384600F0C8FA15B0F0BD70470120E6
:10E6000003F0DABB10B5044800F030FFBDE810405D
:10E61000002003F0D1BB0000EC1C002008B5034A29
:10E6200000924023024AFFF785FF08BD91120200C5
:10E63000182600200A4A012902EBC00007D002294F
:10E6400007D0032907D0042907D0002070470220F3
:10E650007047042070470079704740797047000088
:10E66000CC31020010B5FFF7CAFF04210348FFF7C1
:10E6700039FF02490120487210BD0000F41C00203F
:10E680002DE9F04F8DB0FDF729F818B100200DB03D
:10E69000BDE8F08F7A4C4FF0000BC4F818B4BFF30C
:10E6A0004F8F60680290A568D846284004EB800030
:10E6B00008E021680298814201D86160E6E72840BD
:10E6C00004EB80000C3002A9FEF726FC0028F0D1F4
:10E6D00005AA029901EA050304EB8303491CDB68E0
:10E6E00042F82030401C02910228F2D3059800F035
:10E6F0000300022802D001284ED0A9E0059850223C
:10E70000810D8946B2EB905F00D850210E4666F32A
:10E710009F50059008315B4800F0E7F9070079D079
:10E7200000F02CFA4346082205A9384600F041FAC9
:10E73000029908F1080A2940681A8000001D8642E3
:10E7400023D94F4D0C3530B1C2B204EB8101301AE0
:10E7500090460C3104E02946F2B200259046284646
:10E76000C6B25346384600F024FA0AEB08032DB12E
:10E77000324629464FEA070000F01BFA029909F1D8
:10E78000030001EB900002903BE004EB8101534653
:10E79000324638460C31EFE70598C0F3831006285F
:10E7A00000D30620059960F38911C1F38310801C02
:10E7B00005918100334800F098F9070048D000F037
:10E7C000DDF94346082205A9384600F0F2F908F1C0
:10E7D000080800260FE00298434600EA0501401CA5
:10E7E00004EB81010290042238460C3100F0E1F97B
:10E7F00008F10408761C0598C0F38310B042EAD8EB
:10E8000047B1D4F81054D4F8180468B1384600F071
:10E81000BBF92FE01CE0687A012804D12A68284659
:10E820003946126890476D68002DF4D1384600F0E3
:10E83000ABF98DF800B06846FBF760FBD4F818041C
:10E8400008B9029860609DF80000FBF77BFB11E0BF
:10E85000D4F8104404E02168204689688847646839
:10E86000002CF8D108480221008801EB004007A1E4
:10E8700000F016F8FCF732FF80F0010007E7000017
:10E88000182700204C3202009C1D00204261636B5F
:10E89000656E647320666C757368656400000000C3
:10E8A00000231A4603F02EB908B5012300926A46E8
:10E8B00003F028F908BD1CB5CDE9002302236A4600
:10E8C00003F020F91CBD3EB5069C8DE81C00032317
:10E8D0006A4603F017F93EBD2DE9F0470E46804623
:10E8E0001C46924608293ED894F80C9000202073CC
:10E8F0001946104601F0C6FE0025B54206D218F8AA
:10E9000005201AA12046FFF7F9F903E019A12046D6
:10E91000FFF7F4F96D1C082DEFD317A12046FFF780
:10E92000EDF90025B54210D218F80570FAF79AFDF6
:10E930000068C05D10F03E0F01D03A4600E02E2284
:10E940000EA12046FFF7DAF903E00DA12046FFF7FC
:10E95000D5F96D1C082DE5D301222146504601F062
:10E9600073FE84F80C90BDE8F0870000202530325B
:10E9700078000000202020007C00000025630000BB
:10E9800020000000104810B5FF21816000210160C7
:10E990004160C0F81814C0F8141480F820140B4813
:10E9A00000F0F0F800280DD109480A490A4B401A36
:10E9B000C108002003E000BF23F82000401C88426B
:10E9C000FAD3002010BD0000182700204C320200AE
:10E9D0004C320200CC3102006C1D00200248034979
:10E9E000401AC008704700004C320200CC310200CF
:10E9F00013B56846FEF736FE08B100201CBD02487C
:10EA0000009950F831001CBDCC31020070B50848A7
:10EA10000125D0F8104480F8205405E06572216883
:10EA20002046496888476468002CF7D170BD000013
:10EA3000182700202DE9FF4781460C9D00200C4639
:10EA40002F7B2873984616462946184601F01AFE71
:10EA5000072E42D2DFE806F004090F161F2A3600FF
:10EA600049462846FFF74AF937E0494628462268D2
:10EA7000FFF744F931E0D4E9002349462846FFF77F
:10EA80003DF92AE0A0680090D4E9002349462846D1
:10EA9000FFF734F921E0D4E90201CDE90001D4E91E
:10EAA000002349462846FFF729F916E004F108003B
:10EAB00007C88DE80700D4E9002349462846FFF738
:10EAC0001DF90AE004F108000FC88DE80F00D4E931
:10EAD000002349462846FFF711F9002229464046FF
:10EAE00001F0B2FD2F73BDE8FF872DE9F041858A63
:10EAF00080462D1F4819C01CB0FBF5F0C6B2404639
:10EB0000FEF735FF041E19D000202071012060712E
:10EB1000E58000272546761EC4F800800BE04046BD
:10EB2000FEF725FF60B16179491C617128600546D7
:10EB30007F1CC0F80080B742F1D32046BDE8F081C9
:10EB4000204600F002F80020F8E72DE9F041457971
:10EB500001466B1E002201E00968521C9A42FBD359
:10EB60000F680146002605E038460C68FEF721FFD5
:10EB70002146761CAE42F7D3BDE8F0810121001D8D
:10EB8000FEF7C9BEFEF72DBF10B504460121001DDA
:10EB9000FEF7E7FE10F0FF0F04D12046BDE810405D
:10EBA000FFF7D3BF10BD38B501240094FEF71EFD5A
:10EBB00038BD38B500240094FEF718FD38BD0000BC
:10EBC000064910B500204870091D0860BFF35F8F2B
:10EBD0000349044800F016FA002010BDDC1C002098
:10EBE000302802000C26002010B500F0D9F908B139
:10EBF00041DF10BD20BF40BF20BF10BDFBF7E2B812
:10EC000020B1034909680160002070470E20704759
:10EC10001C2A0200FEB502460E460846FFF7F0FF2A
:10EC2000002868D1002400940194012506208DF865
:10EC30000020ADF8040002948DF8025069462020AF
:10EC4000326869DF2C4F48B100F020FA398802465B
:10EC500005EB014329491846FFF726FE009401946D
:10EC600002948DF8015069464020326869DF40B156
:10EC700000F00CFA02463888214905EB0040FFF706
:10EC800013FE0094019402948DF80040694601201F
:10EC9000326869DF40B100F0F9F902463888194955
:10ECA00005EB0040FFF700FE4FF4B06000900194C8
:10ECB00002946946A120326869DF40B100F0E6F9AC
:10ECC00002463888104905EB0040FFF7EDFD00943F
:10ECD000019402948DF800406946A020326869DFF3
:10ECE00040B100F0D3F902463888084905EB0040EE
:10ECF000FFF7DAFD0020FEBDA41D002068300200F1
:10ED0000B0300200C82F020014300200742F02003D
:10ED10002DE9F0410446D0F8008060DF2168194DEC
:10ED2000074641451CD92888022606EB004016A15B
:10ED3000FFF7B6FD2888424606EB00401EA1236877
:10ED4000FFF7B9FDF006D0F80C012168800200F150
:10ED50000050421A288825A106EB0040FFF7A4FDC9
:10ED6000012467B1384600F091F9024628882AA1AB
:10ED700004EB0040FFF798FD3846BDE8F0812E48CF
:10ED80000470F9E7A41D0020496E73756666696317
:10ED900069656E742052414D20616C6C6F636174C3
:10EDA000656420666F722074686520536F667444D2
:10EDB00065766963652E00004368616E676520743F
:10EDC00068652052414D207374617274206C6F63CA
:10EDD0006174696F6E2066726F6D203078257820BF
:10EDE000746F20307825782E000000004D6178691E
:10EDF0006D756D2052414D2073697A6520666F7282
:10EE0000206170706C69636174696F6E2069732032
:10EE1000307825782E00000073645F626C655F6552
:10EE20006E61626C6528292072657475726E656406
:10EE30002025732E00000000531D002030B514481B
:10EE400091B00078002820D05FF03405ADF8405034
:10EE500010A903A861DF30B1052816D011B0BDE8B4
:10EE60003040FAF7AFBF03AC0A49684600F0CAF871
:10EE700007E000BFD0E9002120469047684600F037
:10EE8000D8F802980028E1D0F4E711B030BD0000B6
:10EE9000531D0020202A0200F8B5134C2078C0B181
:10EEA0000120A07001F0FCFF112814D0022002F014
:10EEB0000FF800258DF800506846FBF71FF811DFAA
:10EEC000064625709DF80000FBF73CF82EB1304651
:10EED000F8BD0820F8BD0020F8BDA57002F0CEFDF9
:10EEE000032001F0F5FFF6E7501D00207CB5204C13
:10EEF000207808B108207CBD0120A070002001F01E
:10EF0000CFFF112819D0002001F0E2FF1948002698
:10EF1000006801908DF800606846FAF7EFFF164927
:10EF200001A810DF05000AD0002020709DF8000025
:10EF3000FBF708F82DB128467CBD00207CBD0120E0
:10EF4000F3E7A67066700721162001F05FFF08B195
:10EF5000FAF738FF0721152001F058FF08B1FAF73A
:10EF600031FF02F0A7FD012001F0B2FFE5E700004C
:10EF7000501D0020B4290200499D01000EB507492B
:10EF8000684600F03FF805E0D0E900108847684681
:10EF900000F04FF802980028F6D10EBDD0290200EB
:10EFA0000148007870470000501D00200548817816
:10EFB00019B1007818B1FFF76FBF08207047FFF74D
:10EFC00095BF0000501D00201FB568464BDF30B1D3
:10EFD000052814D004B0BDE81040FAF7F3BE084984
:10EFE00001A800F00FF806E0D0E900210098904752
:10EFF00001A800F01EF803980028E6D0F4E71FBD32
:10F000003C2A0200016009684160AFF3008010B53E
:10F01000D0E900215368994201D1002104E0D1E9EF
:10F020000034A34202D01946816010BD083141600E
:10F03000F0E7816800290BD0026892680A44826078
:10F0400041684B689A4203D108314160FFF7DFBF46
:10F05000704700000C4A10B502F594730EE0991A3F
:10F06000C91001EBD171491002EBC1010C68844257
:10F0700001D90B4602E005D201F108029A42EED313
:10F08000002010BD486810BD5028020000B5FFF7F1
:10F09000E1FF002800D1014800BD00003C2802002B
:10F0A0004058002800D00120704708B50022425087
:10F0B0004058009008BD000008480068012110F089
:10F0C000010F08D14FF0E020E02280F80024C0F8C2
:10F0D0008012C0F8001102480160704700E100E0B2
:10F0E000180500400649024600200B790BB1852027
:10F0F00070470A6001220A7100224A7170470000BD
:10F10000401C002004490120086004480168C1F344
:10F1100000410029FAD170470C000040180400405B
:10F12000002802D001498001084770475927020092
:10F130002DE9F0418846054600F066FF234E002881
:10F1400028461AD0FCF70AFB304490F848008009A2
:10F15000032802D001280ED007E04FF0A040D0F8DD
:10F160001005E84010F0010F05D003212846BDE846
:10F17000F041FFF775B90221F8E700F051FF0028D0
:10F1800022D02846FCF7EAFA04464FF4807000EBE0
:10F1900084000F4F81B207EB8400D0F8102542F0B5
:10F1A0000102C0F810250846FFF78AF9B8F1000FF0
:10F1B0000AD02846FCF7D2FA56F82000002803D0DF
:10F1C0000120A040C7F80403BDE8F081D42200204C
:10F1D000006000402DE9FC41DFF8BC80044608EBEC
:10F1E0000400002790F930001346C0170E46401C5B
:10F1F00001D008274CE0B0781946C0F34002204601
:10F20000FCF788FA0546401C41D0B078410719D474
:10F21000C0070AD04FF0A04000EB8401D1F80007EE
:10F2200020F00200C1F8000707E0002173782046B3
:10F2300000910A460191FFF7D3F81749204654314F
:10F24000FEF7EFFBB078800718D51448317800EB53
:10F250008500D0F81025124B1A40C0F810254FF445
:10F26000F8524FF4403302EA042203EA01410A4310
:10F27000D0F810150A43C0F8102509E008EB050086
:10F28000327810F8481F41EA8211017000E004272B
:10F290003846BDE8FC810000D42200200060004018
:10F2A000FFE0FCFF4FF0A041D1F81015C14011F074
:10F2B000010000D00120704770B5184D95F8580036
:10F2C00008B1082070BD0020411E2A18401CC0B2A1
:10F2D00082F830102028F8D300242046FCF70CFADE
:10F2E000641CE4B20C2CF8D300240D49E0206C65BA
:10F2F00081F8000401264020891FC1F88002C1F86E
:10F3000000014FF4BE70FFF7DBF80649F007C1F8C3
:10F31000040385F85860204670BD0000D422002008
:10F3200006E000E000600040034890F85800002824
:10F3300000D0012070470000D42200200121B1EB51
:10F34000507F01D101207047002070470020704796
:10F35000704700002DE9F0410546164600790F463A
:10F36000154A00EBC00102EB810494F8201011B1A2
:10F370000820BDE8F081114951F820102868FFF7F6
:10F38000E5FF08B11120F4E739462846FAF7F4FD05
:10F390006660386920601EB1397F2846FDF77CFD24
:10F3A00028680821C0F800150020A061E061012153
:10F3B000606184F82010DCE7302300204C27020035
:10F3C0002DE9F04704460E460079204900EBC000C5
:10F3D00001EB800517463046FFF7B0FF30B12046FD
:10F3E00000F036F820B11120BDE8F0871020FBE7CF
:10F3F0006F61AE604FF49076002731462068FFF7CA
:10F4000054FE4FF4AC7841462068FFF74EFE20686A
:10F41000AA686969C0F84425C0F848152068012128
:10F420008160686878B9B14649462068FFF738FEC0
:10F43000064641462068FFF733FE0643F4D000B18C
:10F440000F27002068613846CEE7000030230020F7
:10F450000079054900EBC00001EB800040690028FD
:10F4600000D0012070470000302300202DE9F04734
:10F4700004460079274900EBC00001EB80072068B3
:10F480004FF00009C0F80095786880B120682249E3
:10F49000C0F8081320680121000B40B200F01F02E1
:10F4A00091404009800000F1E020C0F88011206800
:10F4B000D0F80C25D0F81485D0F80865D0F8105590
:10F4C0004FF0FF31C0F80C15C0F814152068C0F8D3
:10F4D0000815C0F81015501C02D01046FEF7A4FF06
:10F4E000B8F1FF3F02D04046FEF79EFF681C02D0F5
:10F4F0002846FEF799FF701C02D03046FEF794FFB5
:10F500002068FFF725FF87F82090C7F80490BDE832
:10F51000F0870000302300201003020010B590B1E6
:10F52000032814D10A480321008801EB004009A1F7
:10F53000FFF7B6F90220FBF743FF002807D0BDE82C
:10F540001040FAF73FBCBDE8104002F06BB810BDA8
:10F550009C1D002046617374206164766572746935
:10F5600073696E672E0000000078002807D10448F8
:10F570003B21008876DF002801D0FAF723BC7047D2
:10F58000481B002070B502468888C97B00EB400309
:10F5900002EB4304A41D012901D111882180218897
:10F5A0006288914211D9A5DF012568B111280DD0DB
:10F5B000FFF76CFD0246064806A1008805EB0040F7
:10F5C000BDE87040FFF770B9657170BD257170BD01
:10F5D0006C1D002073645F626C655F6761747463A7
:10F5E0005F65786368616E67655F6D74755F72658E
:10F5F000717565737428292072657475726E6564FF
:10F600002025732E000000007CB506468D88C88832
:10F6100005EB450106EB4104A41D172800D2172075
:10F620002188814200D8084660800020207121880E
:10F630002846B5DF50B1FFF729FD02460E480121EB
:10F64000008801EB00400DA1FFF72EF9607900283A
:10F6500010D1F06800280DD01449D1E90201CDE99C
:10F660000001ADF802506088ADF80400F268694608
:10F67000304690477CBD00006C1D002073645F62C3
:10F680006C655F67617474735F65786368616E67EA
:10F69000655F6D74755F7265706C7928292072657D
:10F6A0007475726E65642025732E0000A826020012
:10F6B00048B1064A0168914205D1406804494018A2
:10F6C00002D0012800D0032070470000DEC0ADDE6C
:10F6D00002FEE10E8A7D022A04D90289CB881A44EF
:10F6E000D21C02814289C988511AC91E41817047C2
:10F6F0002DE9F0410D460221904600F58056298003
:10F7000000F10804144F1BE031462046FDF73CF998
:10F7100040B1B8F1000F02D0012288F80020022881
:10F7200016D004E0A0687969884200D978612888F9
:10F7300061880844C01C2880608804EB80040C3475
:10F7400031462046FDF733F90028DDD1BDE8F081D0
:10F750004FF480602880F9E7901C002008B5002154
:10F76000009101460823024A0248FEF73DFD08BD0C
:10F7700070270200581D002008B5002000900448A2
:10F780000823044A01680448FEF72EFD08BD000066
:10F79000B81C002068270200581D00202DE9F05FEA
:10F7A0000025DFF80891DFF808B12C464FF0030878
:10F7B000AA462F46D9F80C0000EB07363046FFF773
:10F7C00077FF78B3012847D0032862D100204FF497
:10F7D000806200BF56F82010491C0ED004EB840153
:10F7E0000BEB8102A8F10100566003221FFA80F89A
:10F7F0000BF82120641CA4B24BE0401C9042E9D3DA
:10F800002C48016879B104EB840102200BF8210037
:10F810000BEB81014E600881254828304480641C30
:10F82000A4B205E007E00221066081804FF0010AE2
:10F8300045F001052DE004EB840100220BF82120A6
:10F840000BEB810101F110024E6030460831FFF7E9
:10F850004FFF45F00205CDE7BAF1000F0CD00220B2
:10F8600004EB8401134A0BF821000BEB81011268B1
:10F870004A60641C0881A4B20E480022011D066083
:10F880003046FFF735FF0B48808802280CD008204F
:10F8900005437F1CBFB2032F8CD3B8F1020F00D2F7
:10F8A0000025E8B2BDE8F09F0420F1E7581D0020D4
:10F8B00034250020B81C002001494978FBF7E6B840
:10F8C000D01B0020002102F0ADB830B585B00C4649
:10F8D00005218DF800101546ADF80200FDF7D2F9AC
:10F8E000ADF804006846CDE90245FCF7D1FA05B051
:10F8F00030BD000070B5054D06460024304655F871
:10F9000024108847641C042CF8D370BDD026020054
:10F910003EB5104D002400BF05EB041002F020FDA1
:10F92000641C022CF8D30124502002210094CDE95C
:10F9300001100849084BB039A02201F1A00000F0E5
:10F94000A9FB08B103203EBD0348401E847000207F
:10F950003EBD000014220020BD1B002000F06CB949
:10F9600000F06CB970B504460025C168184A2846F5
:10F9700002EB00139B688B4202D102EB001003E004
:10F98000401C0228F4DB00202178082904D0092932
:10F9900008D0132914D112E0617A89B980B102F03C
:10F9A000EFFC0DE0617A59B950B100218160817B93
:10F9B00041F00201817307490120087003E001252D
:10F9C0002046FFF797FF2846BDE8704000F0A2BF31
:10F9D00014220020BC1B002000F0E5B908B51388F4
:10F9E0009B0000936B4600F05FF908BD002300F018
:10F9F0005BB938B505460024204609E081782846E1
:10FA000000F080F810B1052800D003240098401CB5
:10FA100000906946284602F08FFC0028EED134B9E8
:10FA2000284600F0C4F910B1072802D0032420466C
:10FA300038BD0724FBE71346002200F069B9000037
:10FA40002DE9F0471F0015460E46814604D0072ECB
:10FA500005D0082E16D102E00E20BDE8F0878DB14A
:10FA6000022D0FD800F0AEF960B14FF0000831461A
:10FA7000484602F047FC041E06D0207BA8420DD069
:10FA80000F20EAE70720E8E7FF214FF6FF7002F0BA
:10FA900039FC041E06D0A0F80090A670607BFF28F9
:10FAA00002D00CE01120D8E72946154800F0C4FA2E
:10FAB000014620466173FF2913D04FF001082573DA
:10FAC000617B0F4800F006FB02000DD0ABB231465F
:10FAD000384600F007FAB8F1000F0ED0082E05D016
:10FAE0000BE002F03DFCDDE70320B6E738886FF05D
:10FAF000050101EB8000796888800020ADE70000F7
:10FB00000422002070B5002402F0FCFB05000BD09D
:10FB1000686820B100F06FF9040000D00324284683
:10FB200002F02EFC204670BD052070BD70B5154654
:10FB30000C46072903D0082C01D0072070BD02F025
:10FB4000E1FB28B105808470BDE8704002F098BBED
:10FB5000052070BD7CB50D46072903D0082D01D0C6
:10FB600007207CBD002602F0CDFB040002D06068B7
:10FB700010B11CE005207CBD617B0F4800F0AAFAA3
:10FB800002004FF00000009001908DF8025010D05C
:10FB9000237B2946684600F03DF9684602F05EFB8B
:10FBA000211D684600F010F90646092801D03046AC
:10FBB0007CBD03207CBD0000042200204FF6FF71B5
:10FBC0004180014909680847B826020030B587B06E
:10FBD0001748FCF7E7FA10B1032007B030BDFCF777
:10FBE00003FA08B18620F8E700F0CEF90020029071
:10FBF0004CF2070403900EE0694604A8FCF79CFA57
:10FC000000988088A0F5404085B204A8FCF754FA1B
:10FC1000284600F075F902AA04A92046FCF773FAF9
:10FC20000028E9D00349012008700020D5E7000032
:10FC30009DBE0100B01B002000F088B900F08CB917
:10FC400070B586B014460E46054600F03BF940B14B
:10FC500005F5404080B20F4A6946FCF754FA40B9B6
:10FC600002E0012006B070BD03A96846FCF764FA03
:10FC700008B10020F6E7A57003984088208004981A
:10FC8000606003988088A0F5404030806846FCF7AB
:10FC900013FAE6E7B41B00200248002141608160AE
:10FCA00070470000B01B0020F0B587B01D46144619
:10FCB00007460E46FF280AD8084600F003F930B17F
:10FCC00003AA3146384600F0E5F840B902E00720C3
:10FCD00007B0F0BD01A903A8FCF72EFA08B1052072
:10FCE000F6E7A67001984088208045B18200286818
:10FCF00090420BD302996068F9F7B8FB01E00298D3
:10FD0000606003A8FCF7D8F90020E1E70420DFE7F2
:10FD10007FB586B01E460D460446FF282AD8A8782F
:10FD200000F0D0F830B304F54040ADF80000A878FA
:10FD300003AA00F54040ADF80200686801902888E9
:10FD40000290A978204600F0A5F80528089813D05D
:10FD500010B108A8FCF754FA694603A8FCF710FA9A
:10FD6000B0B107281DD0082819D00E2817D00320BD
:10FD70000AB070BD0720FBE728B108AA694603A8AE
:10FD8000FCF709FAECE7694603A8FCF700FAE7E795
:10FD90001EB1314603A8FCF7C6F90020E8E71120A0
:10FDA000E6E78620E4E74FF6FF7000F0A9B810B54B
:10FDB000FF2801D9072010BD00F0A8F800F02EF8A8
:10FDC000002010BD00F0F4B870B504460D468078F0
:10FDD00000F078F858B121882846FCF7F9F9002896
:10FDE00004D0072805D0092800D0032070BD0720C3
:10FDF00070BD862070BD01B56846FCF701FA002889
:10FE000000D0032008BD00000149C978FAF73EBEC2
:10FE1000D01B00209BB200F065B8000070B51B4DF0
:10FE20008AB00020687000904FF6FF76019030464F
:10FE300003E0204600F07CF8204600F087F80446F6
:10FE4000B0421DD004F5404080B26A4602A9FCF7DA
:10FE500062F90A28EDD004F5404080B2FCF784F83E
:10FE600008280FD000280BD005461422084905A801
:10FE7000F9F7FCFAADF8184005A80795FFF79EFEC4
:10FE80000AB070BD01206870FAE70000B01B0020C6
:10FE9000BC2602007CB5054616460C46084600F016
:10FEA00011F80020009005F54045019004F540440C
:10FEB000A8B2A1B26B463246FCF71EF9002800D06A
:10FEC00005207CBD07280BD0012809D0082807D0C1
:10FED000052805D0062803D0042801D0002070474B
:10FEE0000120704710B503EB83034FF6FF7404EA5B
:10FEF00003138170DB1C99084260018010BD000073
:10FF00000149FBF783BC00003422002010B50446F1
:10FF1000A0F57F40FF3807D004492046FBF776FC68
:10FF2000A04201D1012010BD002010BD54220020AC
:10FF300010B50446044900F009FE03492046BDE817
:10FF40001040203100F002BE342200200149FDF7AC
:10FF500025BC00005422002070B50A49FDF71EFCA4
:10FF600004464FF6FF7507E000F02CF838B105495C
:10FF70002046FDF713FC0446AC42F5D170BD204687
:10FF800070BD00003422002010B508484021F9F768
:10FF900086FA4FF480742146044800F0A1F9214606
:10FFA0000248BDE81040203000F09AB93422002009
:10FFB000FF2803D80146024800F0C1B9002070476D
:10FFC00034220020FF2803D80146024800F0B7B9C8
:10FFD000002070475422002010B50C46FCF798FB17
:10FFE000FF2804D0024900EB400021F8204010BD5A
:10FFF000642000200068012803D0022801D00020DE
:020000040002F8
:1000000070470120704700000449084490F930000F
:10001000082801DB0120704700207047D42200200F
:100020000449084490F93000082801D201207047A3
:1000300000207047D42200202DE9F0410F46060031
:1000400026D0306820B3706810B3FF2400251CE070
:100050002946706800F04BF948B1FF2C00D12C46BE
:10006000281B401CB8420ED12046BDE8F081FF2C71
:1000700006D108E02146304600F040F8641CE4B2A6
:10008000AC42F7D3FF246D1CEDB2B068A842DFD8B4
:10009000FF20EAE72DE9F0410400DDE90705069EAF
:1000A00016D0A9B1A3B100FB05F7974210D8C21D25
:1000B000B6EBD20F0CD358B155B1E5602160C4E95D
:1000C000013081B2184600F00BF90020BDE8F08144
:1000D0000720FBE770B504000D460DD0206858B12D
:1000E000606848B1FF2D07D000F029F920B1E16820
:1000F000206805FB010070BD002070BD70B50400D4
:100100000D4611D0206800280ED0606800280BD062
:10011000FF2D09D000F013F9002805D029466068AA
:10012000BDE8704000F017B970BD002901D001F0A2
:100130009DBA7047034B1B780BB101F0EBBA082056
:1001400070470000C01B00207CB5044601780020E9
:10015000324D03260E291DD2DFE801F0071C0F1CCB
:100160001D234C5D1C5B1C5D565D28882CA106EB95
:100170000040BDE87C40FEF793BB6088FAF760FC66
:100180000246207A00902888638806EB00402FA161
:10019000FEF799FB7CBD009060886946FFF7C5FFBC
:1001A0007CBD009001909DF80000694620F07E0023
:1001B00040F00100303020F080008DF80000072072
:1001C0008DF8010010208DF802009DF8030040F02A
:1001D00003008DF803009DF8040040F003008DF843
:1001E00004006088E268FFF7A5FF0028D8D0F9F77F
:1001F000E9FD7CBDFBF7DAFE0828FAD00028F8D02C
:10020000BDE87C40F9F7DEBDBDE87C400020F9F791
:10021000F9BC2069F2E7A068F0E700009C1D00200F
:10022000436F6E6E656374656420746F2061207027
:10023000726576696F75736C7920626F6E64656440
:10024000206465766963652E00000000436F6E6E62
:10025000656374696F6E20736563757265643A20B7
:10026000726F6C653A2025642C20636F6E6E5F6838
:10027000616E646C653A20307825782C2070726F3E
:100280006365647572653A2025642E00FBF7DCBD5A
:10029000FBF7DABD10B5FFF799FC88B9FFF738FB1B
:1002A00070B901F0E5F958B901F000FB40B9FCF76D
:1002B000CBF928B9FCF7B0FA10B9FCF753FC08B138
:1002C000032010BD05484FF6FF7181800021816039
:1002D000417001210170002010BD0000C01B0020F2
:1002E000002803D0C91DC908F9F7D9B870470028FC
:1002F00009D001F0070301229A40D2B200EBD100ED
:100300001146FDF703B870472DE9F0410D46060090
:1003100013D0002401270EE004F0070007FA00F0D4
:10032000C1B206EBD400FCF7F1FF10B12046BDE8E6
:10033000F081641CA4B2AC42EED32846F7E740B18A
:1003400000EBD10001F00702007801219140084044
:1003500000D001207047F8B50400C1F3C70501F0D3
:1003600007014FF0010000FA01F0C6B20FD0605D46
:1003700030420CD000208DF800006846F9F7BEFD31
:10038000605DB04360559DF80000F9F7DBFDF8BDF6
:100390002DE9F041044686B001278088FCF7B0FBC8
:1003A0006080207800263F4D082808D0092820D0FA
:1003B0004FF6FF780A2829D00B2853D158E0607AED
:1003C00010B1012809D04DE0A86830B1E168814240
:1003D00003D1AE60A088A88016E06878E8B3A08852
:1003E000A98888423ED1207A06283BD100F076FACF
:1003F00038E0607A88BBA86878B3E168814231D17F
:10040000AE60E868401EE860E6602BE0A878E8B1DE
:100410004046FFF7A5FA4146404517D10846FFF789
:100420009DFA404512D1AE7014216846F9F737F8AD
:100430000C208DF80000ADF80480ADF80280002794
:100440002046FBF701FD6846FBF7FEFC687838B1F3
:10045000A088A988884203D100E003E000F03EFABA
:10046000002F1CD006B02046BDE8F041FBF7ECBCE5
:10047000A8780028F6D0AE7014216846F9F70FF876
:100480000D208DF80000ADF80480ADF80280A06862
:1004900002902046FBF7D8FC6846FBF7D5FC06B077
:1004A000BDE8F081C01B00200349097809B1FCF7C1
:1004B000D5BB082070470000C01B00202DE9FF4F6E
:1004C0002A4883B09946007892468B46B8B14FF6D9
:1004D000FF763046FFF744FA80460020009024481B
:1004E00001AA062100680190CDF808D04046FFF728
:1004F00075FA00256C1E3746072804D017E008203F
:1005000007B0BDE8F08F0520FAE700200090A84270
:1005100001D305464746A04201D20446464640461E
:10052000FFF71EFA804601AA0621FFF757FAD8B155
:100530000528EAD0A8F57F41FF3901D00320DFE785
:100540000399002001B10F80BBF1000F01D0CBF85F
:100550000050BAF1000F01D0AAF80060B9F1000F05
:10056000CED0C9F80040CBE70098D0E7C01B0020F0
:10057000E026020070B5184E86B03078D0B1012068
:10058000B0704FF6FF742046FFF7EAF90546A04227
:100590001DD10020B07014216846F8F780FF0C20B0
:1005A0008DF80000ADF80440ADF802406846FBF756
:1005B0004BFC0EE0082006B070BD00BFFFF774FFD3
:1005C00008B10320F7E72846FFF7CAF90546A54218
:1005D000F4D10020EFE70000C01B0020084A11788A
:1005E00021B1D178032903D3042070470820704734
:1005F000044B43F82100491CD170002070470000D3
:10060000C01B002074220020002801D0FBF71CBC76
:10061000704770B50D00044602D10020F9F7D2FBF7
:1006200014B90020F9F7CEFB287820706988617032
:10063000090AA170A988E170090A2171E88860712E
:10064000000AA07170BD000010B50C46017A0529A2
:1006500008D0407A38B1084808A102682046FDF762
:100660004DFB00E01AB106A12046FDF747FB2046EE
:10067000BDE81040FDF74FBB2C1D00202573000086
:100680000D0A000038B5C3880D46044633B114A0E6
:10069000009015A216A12846FDF730FB217A052906
:1006A0001CD0607A48B1A088FDF7C4FF164951F804
:1006B000202016A12846FDF721FBA0880021FEF787
:1006C00097F903461049207A143951F8202001B0D7
:1006D0002846BDE830400EA1FDF710BB38BD000034
:1006E0001B5B306D000000001B5B313B33316D0044
:1006F00025734C6F67732064726F70706564202877
:1007000025642925730D0A002C1D00202573000087
:100710003C25733E2025733A200000000146054821
:1007200010B50068FDF76DF804461C21F8F7B7FE18
:10073000204610BD60270200014602480068FDF710
:1007400081B8000060270200034802490068FDF7F5
:1007500063B80000D81C0020E8270200F0B5254D42
:10076000254E85B004460027686828B921493068BD
:100770000831FDF75CF8686001460078072817D259
:10078000DFE800F0160408080E0E12002046FCF701
:10079000C1FA02E0204601F07DFE040028D008E006
:1007A0002046FBF7B3F9F8E72046FBF7F7FDF4E73F
:1007B0000F2414216846F8F772FEA4F5E8501D389E
:1007C00000D10024019469466868FBF781FA684605
:1007D000FBF7B8FA07496F60002408313068FDF76D
:1007E0001BF8044801210C30FDF7BBF80028BBD1F1
:1007F00005B0F0BD901C0020602702002DE9F041FB
:10080000234C0025234E207A012730B92248311D80
:100810000068FDF70CF8306038B1022020723168B2
:10082000087928B101281ED116E06560BDE8F08185
:10083000D1E90503C01A4FF48052904200D310460C
:10084000B7EB900F01D2820800E001220869C96865
:100850001844194429DF03E0D1E90301084428DFE3
:1008600058B1112812D003213068FBF77BFA2572AA
:100870006560BDE8F041FFF767BF207C0028D5D157
:10088000BDE8F04100210220FDF75CBC2772CDE7F6
:10089000F8250020D41C0020E827020010B5012113
:1008A0000448FDF744F8002803D1BDE81040FFF7E5
:1008B00055BF10BD9C1C002010B5074C201DFDF736
:1008C00027F8002806D1607C002803D1BDE810403D
:1008D000FFF794BF10BD0000F8250020084910B5AF
:1008E00000231A46A1F10800FFF7E8FD30B1052802
:1008F00004D0002002490C39487010BD0120F9E7EE
:10090000CC1B002010B510461A46F8F7AFFD0020AA
:1009100010BD00002DE9F0471B4F824600263878B5
:1009200086B0002821D00024DFF86080A14600BFF7
:1009300008EB0415A87B810702D410EA0A0F1BD02C
:100940000126284601F09CFCB0B14FF6FF71ADF8CE
:1009500002102988ADF80410862809D007218DF8E7
:10096000001002906846FEF7C5FF06B0BDE8F087AC
:1009700006208DF80000F5E7641C022CD8D3002E69
:10098000F3D187F80090F0E7BC1B00201422002070
:100990002DE9F04707461E481C46154600780E46CE
:1009A00070B185B17CB1DFF86C804FF00009A08890
:1009B00002282BD200EB800118F8210010BB19E0AF
:1009C0000220BDE8F0870520FBE720681FB1818881
:1009D0003A8891420ED11EB101883288914209D1E4
:1009E00080682860206868600A482830008928816B
:1009F0000020E6E7A088214600F05EF80028E4D158
:100A0000C4F80090A088401CA080D0E70A20D8E756
:100A1000B01C002034250020F8B505464068244F5E
:100A20000C46002648B32349CA68824225D8096982
:100A3000814222D3FCF7CAFAF8B128893989884261
:100A40001BD1D5E900018A68904216D10020A7F198
:100A5000280200BF00EB800302EB83035B688B423C
:100A600005D203F580538B4201D9208011E0401C50
:100A700080B20228EED30020F8BD268000960AE05E
:100A8000009829688068884205D100986860388994
:100A900028810120F8BD2088694600F00DF8002863
:100AA000EED12088401C80B220800228E6D3E2E705
:100AB0005C250020581D002070B50E4600EB80011B
:100AC000134800EB81004468306804F5805518B184
:100AD000418800EB810411E0083410E029462046EB
:100AE000FBF752FF20B1012805D0022807D10DE005
:100AF0000120346070BD608804EB80040C3429460A
:100B00002046FBF754FF0028E8D170BD002070BDDF
:100B10003425002038B50C460021009101460423FD
:100B2000074A0848FDF760FB08B10E2038BD064AA9
:100B300004EB840102EB810101200874002038BD20
:100B400064270200581D0020342500200A46FF2893
:100B500003D801461046FFF7FEBB704708467047B2
:100B600070B590B00E4605461C216846F8F797FC14
:100B700000249DF80000039440F002008DF800006E
:100B800001208DF83600019442F654200494059417
:100B90000694ADF834000C94F0798DF83000307A7A
:100BA0008DF831009DF83200142120F00600801CE1
:100BB00020F019008DF8320007A8F8F770FC708952
:100BC0008DF83800000A8DF839000DA807900CA8A0
:100BD00008900220ADF82400ADF828000EA8ADF86A
:100BE00026400B90A88805F10E0307AA6946AADFE4
:100BF00010B070BD1FB501248DF8004000208DF8A5
:100C000001008DF802001849184800F034FBADF8D7
:100C10000400154915481031083000F02CFB8DF800
:100C20000600114911482031103000F024FBADF8C6
:100C30000800BDF80400B0F5407F01D98DF80240EE
:100C400069460B48FAF7F2F900280BD0082809D0BA
:100C5000132807D0112805D043F20141884201D062
:100C6000F9F7B0F81FBD0000001F0020541B002042
:100C7000001E002070B594B00024064607949DF82D
:100C80001C000D4620F00F00401C20F0F00010303A
:100C90008DF81C0008798DF81D009DF81E001C21A0
:100CA00020F00600801C8DF81E006846F8F7F7FB60
:100CB0009DF80000019440F010008DF8000007A896
:100CC000CDE9044001208DF84E00039442F65320F4
:100CD0000694ADF84C000D9468798DF83400A8792D
:100CE0008DF835009DF83600142120F00600801C98
:100CF00020F0180040F001008DF8360008A8F8F741
:100D0000CEFB13A808900DA809900EAA05F10C01BE
:100D1000304600F010F8ADF828001420ADF82C0093
:100D20000EA8ADF82A400C90B088B31D08AA6946F9
:100D3000AADF14B070BDF0B58C885470240A064642
:100D400094708879D070347E00230420E40707D0A3
:100D50000C782CB10C891471240A012354710620DB
:100D6000347EA4070DD54C785CB11518CC682C7076
:100D7000270A6F70270C240EAF7043F00203EC704B
:100D8000001D347E640703D5897809B143F004035C
:100D90001370F0BD70B5012670044FF0E0210025FE
:100DA000C1F88001084C4010C4F84803C4F8080397
:100DB00066602F20FEF7B4F9A660044C2F20A560D2
:100DC000FEF7AEF9A57070BD00100140681C002050
:100DD0001FB501238DF800308DF808100192D0E97D
:100DE0000012684690471FBD10B504460648417979
:100DF0002046F9F74BFE002804D12046BDE81040FC
:100E000000F088BA10BD0000981B002070B50D4698
:100E10000446F8F765FE70B12846F8F773FE68B12E
:100E20006807000E002C0CDA04F00F0101F1E0213C
:100E300081F8140D09E042F2010070BD42F2020097
:100E400070BD04F1E02484F80004002070BD0000AF
:100E500038B50021012548B101280CD0032809D15B
:100E6000FEF72AF9BDE83840FCF710BF4FF0E0204C
:100E7000C0F8805138BD8DF800106846F9F73EF88B
:100E8000064C207808B9FCF7E5FEE068401CE060FD
:100E9000A5709DF80000F9F755F838BDC022002074
:100EA0003EB5044609496846FEF7ACF808E000BFC5
:100EB000D0E900212046904730B16846FEF7B9F8E6
:100EC00002980028F4D13EBD11203EBDB829020091
:100ED0003EB5044608496846FEF794F807E000BFAF
:100EE000D0E90021204690476846FEF7A2F8029814
:100EF0000028F5D13EBD0000C42902002DE9FC41C7
:100F000004460C3000278046FBF7CCFE4FF6FF75F9
:100F10000646A842208803D1FBF7B4FE064602E04D
:100F20003146FBF799FE20880022012100F0C6F827
:100F3000AE4212D06A4607213046FEF757FD60B92F
:100F4000019D95F844003435C00705D1414605F1AF
:100F50001200FBF76CFE00B12F46002320881A46D2
:100F6000394686DF05000BD0002320881A4631461B
:100F700000F088F82088294600F002F9BDE8FC81DD
:100F8000002FFBD1002320881A46314600F07AF862
:100F90002088002241F20601FAF76EFEEEE700001B
:100FA0002DE9FC411D46089C16460F46804644B17B
:100FB0006B46012207213846FEF742FD112801D079
:100FC00010B10320BDE8FC8150210198F8F767FAC1
:100FD000019806700198E56034302060019818305F
:100FE00020610198401C60610748E061019940461A
:100FF0001131FBF709FD0028E3D107213846FEF740
:10100000A9FD0528DDD0DDE780220020002835D0AD
:101010000278910701D411062FD4C2F302110429DA
:101020002BD8930703D5032901D1110625D5437881
:1010300081788B4221D8072B1FD310291DD8C17866
:101040004B071AD40079430717D40B0715D40307AD
:1010500013D4D2074FEAC17201D042B10FE062B996
:1010600089070AD4C10708D1800706D407E0890799
:1010700005D4C10703D1800701D4002070470120A7
:101080007047000070B50C4605466AB1002B12D0BF
:1010900009480122C1782846F9F710FD2146284663
:1010A000BDE87040FBF7D8BD002B04D0BDE8704010
:1010B0000846FBF7D3BD70BDD01B0020F0B5174D1F
:1010C00014460F460A4685B006462978F9F7F6FC1D
:1010D000002F1FD00CB1012200E0002269783046B9
:1010E000F9F7ECFC012C17D00022A9783046F9F76B
:1010F000E5FC0022E9783046F9F7E0FC14220849C3
:101100006846F8F7B3F9ADF802608DF80840684614
:10111000FAF7B0FE05B0F0BD0122E6E7D01B0020D3
:10112000F426020010B586B0044614216846F8F78C
:10113000B6F904208DF80000ADF802406846FAF7D1
:1011400099FE06B010BD000002498969002900D04F
:1011500008477047D01F002030B585B00C460546C3
:10116000142206496846F8F781F9ADF8025068463E
:101170000294FAF75BFE05B030BD0000382602008D
:1011800030B585B00C460546142206496846F8F786
:101190006DF9ADF8025068460294FAF76BFE05B09F
:1011A00030BD00000827020070B51D4851210160C4
:1011B000642141600121816001730146194800F0FA
:1011C0004FF8174880211030002401604FF4D0619F
:1011D00041604FF4C07181600473014611480830CA
:1011E00000F03EF80E482821203014250160A0218F
:1011F000C0E90115047301460A48103000F030F8C8
:1012000007487D213030C0E9005105218160047319
:101210000146BDE870400348183000F021B80000D6
:10122000F01E00204C1B002010B503680A68896876
:101230009C1A8C4202D9591A016010BD012102602A
:10124000017110BD10B54B68026889689C1A8C4208
:1012500002D91144016010BD00210360017110BD6D
:101260000A7B1AB149680160002102E00968016047
:1012700001210171704710B504460079002820460D
:1012800002D0FFF7DFFF01E0FFF7CEFF206810BDBF
:1012900010B5094C0020D2B2207004F10800FEF70E
:1012A0008FF808B1F8F78EFD6078002802D0217819
:1012B0000029FAD010BD0000E41C002003480022E1
:1012C00001490079F9F7A6BBE90D0200981B00203F
:1012D0007CB50E490E4C0022D1E90001CDE9000198
:1012E0006946A088FEF7A7FB4FF6FF7507E00846A2
:1012F000FEF736FBA08000226946FEF79CFBA18822
:10130000A94201D01128F2D17CBD00008C26020038
:10131000A41B002070B586B0064601250024FBF70B
:1013200017FB112812D005DCF0B1062828D00828B8
:1013300008D125E0A0F54051023907D0A1F5407150
:10134000FF3924D001463046FFF706FF2A46124DEA
:1013500030462979F9F7B2FB697906B02246304662
:10136000BDE87040F9F7AABB14220C496846F8F7AB
:101370007DF8ADF8026001246846FAF757FDE5E70D
:1013800000253046FBF77EFCFBF738FADEE73046F7
:10139000FBF780FFDAE70000981B002060260200C0
:1013A0002DE9F0410746806A14468846C8B30025F7
:1013B00031E000BFB96A05EB450001EB8006B0885B
:1013C000801CFE2802D90C20BDE8F0812288401C38
:1013D00008F8020020881622401C80B2208008F8FD
:1013E00000202088401C80B2208000EB080130885B
:1013F00000F09CFD2188084480B22080B28842B170
:10140000B16871B14044F8F731F82088B1880844D8
:1014100020806D1CEDB297F82C00A842CAD800209D
:10142000D2E7FFE70720CFE730B5A7B069481D90A6
:1014300000241DA96848FCF790FB08B1F8F7C2FC2E
:101440001C216846F8F72BF80520ADF80A009DF836
:101450000400012520F00F00401C20F0F0001030A7
:101460008DF804009DF805008DF80C5020F0FF0069
:101470008DF805009DF80600009420F0FF008DF81F
:1014800006009DF807008DF80D4020F00F00401C6D
:1014900020F0F00010308DF807009DF808008DF85E
:1014A0000E4020F0FF008DF808004B48ADF81440C6
:1014B0006946E438F9F794FD08B1F8F783FC142184
:1014C00017A8F7F7ECFF9DF86900179420F00F00BC
:1014D000401C20F0F00010308DF869009DF86A0083
:1014E0008DF8605020F00F00401C20F0F00010300C
:1014F0008DF86A009DF86B00199420F0FF008DF8BC
:101500006B009DF86C0017A920F00F00401C20F024
:10151000F00010308DF86C0064208DF868002E48C3
:10152000F838F9F7E5F908B1F8F74CFC2BA04021A1
:101530000068269007A8F7F7B2FF29A107A8F9F7D6
:10154000D3FD2CA109A8F9F7CFFD2CA10BA8F9F721
:10155000CBFD2DA10DA8F9F7C7FD2DA10FA8F9F717
:10156000C3FD2DA111A8F9F7BFFD59200021CDE938
:101570001E012B48209026A8249004208DF894006A
:101580008DF888505920ADF88A00ADF88C500220B3
:10159000ADF88E001EA8139024A8149022A81590D0
:1015A0009DF8580020F00F00401C20F0F000103093
:1015B0008DF858009DF8590020F0FF008DF8590073
:1015C00007A8F9F7D5FA002801D0F8F7FBFB27B0F8
:1015D00030BD0000FDEB0100E41E0020000102030D
:1015E0004E6F7264696353656D69636F6E64756392
:1015F000746F72004E52463558000000543031333B
:101600003938333600000000323031362E343200A3
:10161000302E312E32000000312E322E33000000E9
:101620005634120010B50020F9F7CAFE08B1F8F7D9
:10163000C9FBF9F71FFE08B1F8F7C4FB33DF002838
:1016400003D0BDE81040F8F7BDBB10BD10B500F0E9
:10165000ABF80548002203494078BDE81040F9F78F
:10166000D9B9000071D10100D81B002000F016B9D3
:1016700010B51148FAF7FBFD0F48401CFAF7F7FDCB
:101680000D48801CFAF7F3FD0B48C01CFAF7EFFD7C
:101690000948001DFAF7EBFD0748401DFAF7E7FD82
:1016A0000548401E8179182903D00121C17100200D
:1016B00010BD032010BD0000D91B002010B500781C
:1016C000114C0A2813D004DC082810D009281AD19C
:1016D0000DE00B280BD0132815D100220B49A0795F
:1016E000F9F798F900220A49A078F9F793F900224E
:1016F00006496079F9F78EF96078BDE8104000225C
:101700000349F9F787B910BDD81B0020C5F80100BF
:1017100071D1010070B50D467AB114467DB108460D
:10172000FFF774FC68B12868606028792072201D7A
:10173000206001206072002070BD0E2070BD00206E
:10174000F6E7072070BD000010B5044600780528B4
:1017500002D0122821D105E06088A168BDE81040C0
:1017600000F060B90F480021806880B10D48237AED
:101770001030007800F0010203B101239A4206D331
:10178000627AC0F3400002B10122904200D20121EE
:10179000608801230022FBF749FC2046BDE8104089
:1017A000FAF776BBD81B002030B50446008885B018
:1017B00014284FD00ADC11282CD0132828D134F853
:1017C000040FF9F73DF901282FD038E0192847D048
:1017D0001A281DD1A088FEF76FF8002818D1A0881C
:1017E000F9F708F90028A0884BD02A490022097887
:1017F000F9F764F902208DF80000A088ADF8020026
:1018000000208DF808008DF809006846FAF732FBD1
:1018100005B030BD207A3D2804D04FF48851A0880F
:10182000002224E041F23D01F9E72079C00701D010
:10183000012200E0022220880121FFF73FFC34F85A
:10184000045B142214496846F7F710FEADF8025005
:101850000294DAE705B0201DBDE83040FFF74EBB2B
:10186000217A201D41B14279008802F0030205B0BF
:10187000BDE83040FBF736BC05B0BDE83040F8F7B6
:10188000C1BB05B00122BDE8304041F20601FAF7C4
:10189000F3B90000D01B0020302702000A7802496B
:1018A0000979F9F70BB90000D01B002010B51448D6
:1018B000FAF7D4FC1248401CFAF7D0FC1048801C00
:1018C000FAF7CCFC0E48C01CFAF7C8FC0C48001D07
:1018D000FAF7C4FC0A48017818290FD04178182972
:1018E0000CD08178182909D0C178182906D001793F
:1018F000182903D001214171002010BD032010BD23
:10190000D01B002070B50C460546F9F799F8012860
:1019100002D043F2020070BD21004FF00000FAD067
:1019200028467EDF70BD00002DE9F74F8AB0924651
:1019300088460A98F9F784F806464FF6FF7900249E
:101940004D4627460A98FEF75FFA8346202101A8F4
:10195000F7F7A5FD012E01D0DEB105E02F480022EA
:1019600001790A98F9F7AAF8B8F1000F16D098F89B
:101970000000C00714D00A98FBF784F905464845D3
:1019800016D1FEF729F8054648450ED04FF0010B59
:101990000CE043F202000DB0BDE8F08F852721E096
:1019A0001F48CDF810A008901CE003246CB121E082
:1019B000012E0AD10A98F8F773F930B90A98FFF79F
:1019C000B1FB0A98F8F76CF950B101A800905346A2
:1019D000324629460A98FFF7E3FA040002D009E0EC
:1019E000852712E0012E10D001AB002239460A985B
:1019F0007FDF044654EA07000DD000225B462946EB
:101A00000A98FFF73FFB2046C5E701AB424639463F
:101A10000A987FDFEDE70122F0E70000D01B0020ED
:101A2000802200203EB505460C466846FBF7ACFE1A
:101A30006A4621462846FDF748FF09480099C268D2
:101A40002846FFF771FF0446014601222846FAF7AF
:101A50002BFC21462846009AFAF7AEF93EBD00005D
:101A6000D81B0020002805D1034901204870002020
:101A7000F9F7E8BE70470000C022002010B516201C
:101A8000F8F72EF848B10A4882684FF4800152B145
:101A9000016821F48001016010BDBDE8104042F2F0
:101AA0000100F8F78FB94FF0E020C0F8801110BDA9
:101AB0008024002010B51620F8F712F880B10F48E6
:101AC00090F800044009F8F71DF860B10C488268EE
:101AD0004FF480016AB1016841F48001016010BDDA
:101AE00042F2010001E042F20200BDE81040F8F7C6
:101AF00069B94FF0E020C0F8001110BD16E000E019
:101B0000802400202DE9F84F204D92468946064654
:101B10009846012269461846AF68F9F787FD58B321
:101B2000009800210446801C09E000BF00EA07037A
:101B30005AF8212005EB8303401C491CDA6041451B
:101B4000F4D34FEA164AFAF76DF84AEA0041601CEE
:101B5000384005EB80003C4005EB8402C160D06852
:101B600066F3C50068F3891069F39F2020F0030035
:101B7000401C20F00400D06095F8200402E000BF73
:101B8000FCF77EFD0028FBD1BDE8F88F1827002068
:101B900070B50C00054602D10020F8F713F915B90D
:101BA0000020F8F70FF9207828702088000A687064
:101BB0002068000CA8702068000EE8702079287159
:101BC000207A68712089000AA871A068000CE87169
:101BD00070BD00002DE9F84F1D4C00256846D4E982
:101BE00001A6FAF729F8002738B30023009A6168A4
:101BF0001CE0D1F800C00846944503D9ACEB0202C2
:101C00000A6015E0A2EB0C0263440760D0F80CC038
:101C1000C1698146BCF1000F08D006EB030828F02B
:101C20007F48C0E9018CC9F81C5005460029E0D165
:101C300028466160FBF7B2FA03E02846FBF7AEFAEC
:101C400010B15046F9F720FEE770BDE8F88F0000AC
:101C5000681C00200D4B10B5596831B102680C6842
:101C6000A24204D8A21A0A60C161586010BD0B4696
:101C700003E00B46C969121B21B10C689442F8D3EA
:101C8000A41A0C600260C161D86110BD681C0020FC
:101C90002DE9F041144E77683D462C4603E084421E
:101CA00004D02546E469002CF9D11BE0D4B1A5424B
:101CB0000BD1F869706040B90C490120886000219F
:101CC000B160F0702F20FDF72BFA2168E069E86120
:101CD00010B10268114401607068874202D001208F
:101CE000BDE8F0810020FBE7681C002000100140E7
:101CF0007CB5064600240D468DF800406846F8F78E
:101D0000FDF801A800F0E4F970B1057009494660DA
:101D10009DF8040048709DF80000F8F713F91420AE
:101D2000F7F7F2FC20467CBD04249DF80000F8F78C
:101D300009F9F7E7742300202DE9F041194D6C688B
:101D4000002C2CD0184800270068A968B846401A13
:101D500020F07F462068B0420CD82146361A07444E
:101D6000E469087C20B181F8108088694969884756
:101D7000002CEFD129786878814206D1401CC0B28E
:101D80006870022801D185F80180064869780C3016
:101D900040F82170BDE8F0411420F7F7B5BCBDE86C
:101DA000F0810000681C0020041501400149012059
:101DB00008707047E41C002010B588B0044620224B
:101DC0000E496846F7F752FB06200090C01F0190AD
:101DD000029003904FF0EB7006900CB1084A00E0BF
:101DE000002269460748FBF769FF08B1F7F7EAFFE9
:101DF0000448001F447008B010BD00008429020090
:101E0000AD1D0200E81C00201FB50A4601788DF8C0
:101E1000001041680191017A8DF80810C0680390A4
:101E2000044850F82210001F50F8222068469047BE
:101E30001FBD00003C1C00202DE9FF410C464FF463
:101E4000927705463946FDF72BF90026C0B1394691
:101E50002846FDF72AF902208DF80000D5F8800405
:101E6000C5F880040390D5F83C058DF80800E068BB
:101E70000190A661E661D4E900126846904723E02C
:101E80004FF4887739462846FDF70AF9E0B139461C
:101E90002846FDF70AF9D5F83C15A069884213D108
:101EA000E06960B1E268D5F8000220F02000C5F8D2
:101EB0000002E069A0612069E661E06001E0A661DE
:101EC000E2682046FEF784FF4FF4A27739462846A1
:101ED000FDF7E6F860B139462846FDF7E6F8A06957
:101EE00030B1A661D5F83C152046E268FEF770FFD8
:101EF0004FF4907739462846FDF7D2F8002813D0E2
:101F000039462846FDF7D1F8606900280CD0D5F88D
:101F10004C058DF800608DF80800A068019066619E
:101F2000D4E9001268469047BDE8FF810870000AB6
:101F3000487002207047000010B514210448F7F7DC
:101F4000AEFA04480068FBF741FC002010BD000019
:101F5000F8250020E82702002DE9F05F8346DDE93F
:101F60000A4A994690460D460846012703E000BFFD
:101F7000B0FBF8F07F1C4045FAD2B94500D94F4676
:101F80005FEACA7012D18CB15FEA8A7002D5B9F1EA
:101F9000000F01D0202607E0302605E031465846E4
:101FA000641EF9F78BFB0CB1A742F7D35FF0010673
:101FB000B9F1010F02D9A9F1010903E0B5FBF6F06F
:101FC000404502D306FB08F6F2E7DFF83C9000BF7D
:101FD000B5FBF6F000FB165519F800105846F9F756
:101FE0006DFBB6FBF8F6002EF2D15FEACA7009D09D
:101FF000002C07D0A74205D220215846641EF9F7CD
:102000005DFBF5E7BDE8F09F78270200034800225A
:1020100001498078F8F7FEBC8DBA0100981B0020BA
:10202000F8B5054680B2FAF7D9FE040013D0154E74
:10203000207A0027317B88420ED2A8B204F10A012F
:1020400075DF28B1112806D0BDE8F840FFF77CB84D
:10205000207A401C2072F8BD2772307C38B1A8B2BB
:102060003B2176DF18B1082801D0FFF76DF87169C0
:102070000029F0D08DF80070ADF80250684688470E
:10208000F8BD0000D01F0020417939B190F8B2109E
:1020900021B990F8B40008B10120704700207047C2
:1020A00001460148FBF719BCEC1F002030B4044680
:1020B000007A00280AD06088002166DF28B1112844
:1020C00002D0616830BC08470120207230BC7047E4
:1020D0000A494A788B78521CD2B2934200D100222E
:1020E0000B78934201D1002070470270487800EBD2
:1020F000400001EBC000001D704700007423002069
:102100002DE9FC411646DDE90854CDE900541F468F
:102110008046022200F00CF8002807D1CDE90054D7
:102120003B4610223146404600F002F8BDE8FC81F3
:102130002DE9FC5F0026DDE90C4B994692468E4660
:1021400080462788354630E0D8F80400002200EBAE
:10215000850069460068019001A864DF002830D13D
:102160009DF8000050451FD10EB1002100E0022172
:10217000228808441118594522D846B9521C90B2F9
:10218000208009F800E02088401C2080012621885A
:1021900001A801EB0902694664DF002811D12088FB
:1021A0009DF80010084420806D1CB8F80000A8427B
:1021B000CADC56B12088C01B401E80B2FF2802D95D
:1021C0000C20BDE8FC9F09F807000020F9E710B5D6
:1021D000042817D209B1032400E00024F8F798FF7F
:1021E0004FF0A04101EB8000D0F8001721F44031FE
:1021F000C0F80017D0F8001741EA0441C0F80017F2
:10220000002010BD062010BD002070472DE9F84FBA
:10221000114D884681461E4617466946DDF828A0BE
:102220002868FBF7EEFA040013D01C21F7F737F902
:1022300000202071C4F80090C4E90486C4E902A714
:1022400069462868FBF7FEFAFEF736FB0020BDE87A
:10225000F88F0420FBE70000E827020082780121C4
:10226000012A0BD0062A09D0072A06D0082A06D14F
:10227000416889880931890800E01421018070478C
:102280001CB50446002000900190A0788DF8020053
:10229000617B1A48FDF71EFF020017D0237BA1784F
:1022A0006846FDF7B7FD6846FFF7D8FF208804F1C0
:1022B000080369466268FDF72BFD48B1072806D080
:1022C00001210F4A112808D086280FD003201CBDF9
:1022D000A17B21F00301A1731CBDA07B20F00100B4
:1022E00040F00200A073117000201CBDA37B23F0FE
:1022F000020343F00103A37311701CBD04220020EC
:10230000BC1B002038B505460C46002001E00098B3
:10231000401C00906946284600F00EF800280AD0BC
:102320008178A142F3D1817B8A07F0D4C907EED12D
:1023300081680029EBD138BD10B5084B0A6809E067
:1023400003EB02142488844203D103EB02100A60D9
:1023500010BD521C022AF3D3002010BD142200200D
:102360004FF6FF710180FF2181704173817B21F065
:102370000301817300210173416081607047000097
:1023800070B50546002406E0687B2044C1B20648CB
:10239000FDF7B4FE641C287BA042F5D82846BDE8B2
:1023A0007040FFF7DDBF0000042200202DE9FC474C
:1023B000064636489846144600780D464FF0000908
:1023C00078B37DB32888A0F57F41FF3931D0688884
:1023D00048B36868FAF7FAFD68B374B32088ADF8BB
:1023E0000000678801A8FEF799F904002FD084F84F
:1023F00000804FF0000A84F816A0BDF80000A0820B
:1024000068682061214801210C38FBF784FAE060FC
:10241000288820816888A080E780B8F1030F1DD04C
:1024200020E001E003E004E00220BDE8FC87052095
:10243000FBE70420F9E70320F7E7FFE7288969466F
:1024400087B2384600F0ACF80028EED1CAE7BDF8F4
:102450000010384600F098F80820E6E70420A07540
:102460003068A061A4F80A9001A8FEF765F946B1AA
:10247000C6F804A0E1680648316086F80AA0008921
:102480003081FEF70BFA0020CFE70000B01C0020DF
:102490005C2500202DE9F8430D46898A374A01EB77
:1024A000810102EB810630B129463046FDF712F971
:1024B0000120BDE8F88331897068002400EB8107B2
:1024C0002E48A97DA8384FF00E0807294ED2DFE824
:1024D00001F00D2D162404404A004460A9690160F2
:1024E00026482749A838FEF797FA30B10220A87588
:1024F000042339462A1D009423E00A20D9E72869DD
:102500002A4608B1032000E001209075042305F15C
:102510000C0207F10801009413E00120A875009453
:10252000E88807F10C0183002A690AE028782A4626
:1025300003280CD006209075042305F10802391DEC
:1025400000941048FBF750FEA8B144460FE0052068
:10255000F1E70621A9750A4940680988FEF7DAFA09
:10256000040004D107E041F61D5400E00F24294681
:102570003046FDF7AFF820469BE7000034250020E9
:10258000901C0020581D002001EB8102034901EB43
:1025900082014A89101AC01E4881704734250020E4
:1025A00070B5C01C82B240F2FE30824201D30920D5
:1025B00070BD114B00204FF4806500BF00EB80041C
:1025C00013F8246096B903EB8406348976891444A1
:1025D0003444A4B2AC4209D2088000EB800003EB83
:1025E0008000418911444181002070BD401C80B2AF
:1025F0000228E3D3072070BD34250020AC1D002045
:10260000CC1D0020111213140D0E0F10301F0020CE
:10261000501F00207C1F00200D00030095B2010018
:102620000E00030095B201000F00030095B20100F7
:102630001000030095B20100070000000000000038
:102640000000000000000000000000000600000084
:10265000000000000000000000000000000000007A
:10266000100000000000000000000000000000005A
:102670000000000011000000000000000000000049
:102680000000000000000000010000000100010047
:1026900088260200010001009C26020000000000C4
:1026A0009102020019C60100770A00000000000034
:1026B000770A00000000000065F901000700000033
:1026C000000000000000000000000000000000000A
:1026D00091030200BD16020019C9010099C601004C
:1026E000010000000000000001000600CC1B0020DB
:1026F0004917020001000000000000000000000077
:1027000000000000000000000700000000000000C2
:1027100000000000000000000000000003000000B6
:1027200000000000000000000000000000000000A9
:102730000500000000000000000000000000000094
:10274000000000000906020000000050B19A0100DC
:1027500003000000542300200738FDD87047000014
:102760007C1C00200000FFFFDEC0ADDEFF011EF17B
:10277000DEC0ADDEFE011EF1303132333435363786
:1027800038394142434445466E72665F6673746FE2
:10279000726167655F696E6974006E72665F667309
:1027A000746F726167655F756E696E6974006E72D1
:1027B000665F6673746F726167655F7265616400FE
:1027C0006E72665F6673746F726167655F77726958
:1027D0007465006E72665F6673746F726167655FC1
:1027E0006572617365000000C01C002000100000CD
:1027F0000400000001000000E1CC0100391F0200CC
:10280000050902000D22020085BC01005D0B0200DB
:102810000922020065CF0100000000000000000056
:1028200000000000000000000000000000000000A8
:10283000182802003028020004000000556E6B6E5C
:102840006F776E206572726F7220636F646500002F
:1028500000000000982E020001000000442D02003C
:1028600002000000382B020003000000B82D020017
:10287000040000000C2E020005000000EC2C0200F9
:1028800006000000882C020007000000F42D020062
:1028900008000000002D020009000000642D020065
:1028A0000A000000802E02000B000000202B020016
:1028B0000C000000182D02000D000000E82E0200A0
:1028C0000E000000E42D02000F000000202E020088
:1028D00010000000542E020011000000FC2E020027
:1028E00012000000D02E0200130000006C2E020027
:1028F00080000000A02C020081000000DC2B020000
:10290000820000009C2B0200830000007C2B020050
:1029100084000000B82B020085000000C42C0200D7
:1029200086000000CC2D020090000000682C020000
:10293000910000005C2B0200920000002C2D020090
:1029400000820000342E020001820000802D02006F
:10295000028200009C2D020000840000F82B02007F
:1029600001840000A42E020002840000402C02001A
:10297000038400001C2C02001DE6010005E6010096
:10298000FDE50100FFFFFFFFFFFFFFFFFFFFFFFF70
:10299000FFFFFFFF00000000000000000000D60164
:1029A00007000000B4320200BC3202000000000048
:1029B0000000000001000007A4290200B429020061
:1029C00008000000DC290200EC29020008000000D9
:1029D000EC290200FC29020008000000E432020099
:1029E000F43202000000000000000000D4320200B7
:1029F000E432020000000000000000006432020027
:102A00006C3202006C3202009432020094320200F6
:102A1000AC320200AC320200B4320200481B00208B
:102A2000FC2902001C2A020008000000BC3202003F
:102A3000CC320200CC320200D43202002C2A020036
:102A40003C2A020008000000004040404040404056
:102A50004040414141414140404040404040404071
:102A60004040404040404040400502020202020215
:102A70000202020202020202022020202020202064
:102A80002020200202020202020290909090909078
:102A90001010101010101010101010101010101036
:102AA00010101010020202020202888888888888AA
:102AB0000808080808080808080808080808080896
:102AC000080808080202020240000000492A020029
:102AD000616464725F69735F77697468696E5F626D
:102AE0006F756E647328705F66732C207061676504
:102AF0005F616464722C20286C656E202A20705FF0
:102B000066732D3E705F666C6173685F696E666F99
:102B10002D3E65726173655F756E697429290000C9
:102B20004E52465F4552524F525F494E56414C49B4
:102B3000445F4441544100004E52465F4552524F5B
:102B4000525F534F46544445564943455F4E4F5498
:102B50005F454E41424C4544000000004E52465FE6
:102B60004552524F525F464541545552455F4E4F74
:102B7000545F454E41424C45440000004E52465F72
:102B80004552524F525F4D555445585F554E4C4F2C
:102B9000434B5F4641494C45440000004E52465F5E
:102BA0004552524F525F4D555445585F4C4F434B21
:102BB0005F4641494C4544004E52465F4552524F94
:102BC000525F4D555445585F434F4E445F494E49FF
:102BD000545F4641494C4544000000004E52465F58
:102BE0004552524F525F4D555445585F494E4954D6
:102BF0005F4641494C4544004E52465F4552524F54
:102C0000525F424C455F495053505F52585F504BA2
:102C1000545F5452554E4341544544004E52465F12
:102C20004552524F525F424C455F495053505F509E
:102C30004545525F52454A45435445440000000013
:102C40004E52465F4552524F525F424C455F49508B
:102C500053505F4C494E4B5F444953434F4E4E4592
:102C600043544544000000004E52465F4552524FC7
:102C7000525F4150495F4E4F545F494D504C454D56
:102C8000454E5445440000004E52465F4552524F57
:102C9000525F4E4F545F535550504F52544544006D
:102CA0004E52465F4552524F525F4D4F44554C4530
:102CB0005F4E4F545F494E495449414C495A45442F
:102CC000000000004E52465F4552524F525F4D4F3A
:102CD00044554C455F414C52454144595F494E492A
:102CE0005449414C495A4544000000004E52465F49
:102CF0004552524F525F4E4F545F464F554E44001F
:102D00004E52465F4552524F525F494E56414C49D2
:102D1000445F5354415445004E52465F4552524F12
:102D2000525F444154415F53495A45004E52465FF9
:102D30004552524F525F494F5F50454E44494E47AE
:102D4000000000004E52465F4552524F525F5356AC
:102D5000435F48414E444C45525F4D495353494EA1
:102D6000470000004E52465F4552524F525F494E57
:102D700056414C49445F4C454E47544800000000C2
:102D80004E52465F4552524F525F4452565F54571F
:102D9000495F4552525F414E41434B004E52465FA0
:102DA0004552524F525F4452565F5457495F455205
:102DB000525F444E41434B004E52465F4552524F84
:102DC000525F494E5445524E414C00004E52465FB0
:102DD0004552524F525F53544F524147455F4655FB
:102DE0004C4C00004E52465F4552524F525F4E557A
:102DF0004C4C00004E52465F4552524F525F494E76
:102E000056414C49445F504152414D004E52465F3D
:102E10004552524F525F4E4F5F4D454D00000000EE
:102E20004E52465F4552524F525F464F52424944BE
:102E300044454E004E52465F4552524F525F4452F7
:102E4000565F5457495F4552525F4F56455252554F
:102E50004E0000004E52465F4552524F525F494E5F
:102E600056414C49445F4144445200004E52465F33
:102E70004552524F525F5245534F555243455300AE
:102E80004E52465F4552524F525F494E56414C4951
:102E9000445F464C414753004E52465F53554343AF
:102EA000455353004E52465F4552524F525F424C7B
:102EB000455F495053505F4348414E4E454C5F413A
:102EC0004C52454144595F45584953545300000002
:102ED0004E52465F4552524F525F434F4E4E5F43F4
:102EE0004F554E54000000004E52465F4552524F1F
:102EF000525F54494D454F55540000004E52465FB5
:102F00004552524F525F4255535900007761726EDD
:102F1000696E670064656275670000001B5B313B8A
:102F200033306D001B5B306D000000001B5B313BDC
:102F300033316D001B5B313B33326D001B5B313B2A
:102F400033336D001B5B313B33346D001B5B313B16
:102F500033356D001B5B313B33366D001B5B313B02
:102F600033376D00696E666F000000006572726F26
:102F70007200000073645F626C655F6366675F7315
:102F8000657428292072657475726E6564202573D6
:102F9000207768656E20617474656D7074696E6702
:102FA00020746F2073657420424C455F4741545430
:102FB000535F4346475F534552564943455F434835
:102FC000414E4745442E000073645F626C655F6349
:102FD00066675F73657428292072657475726E6503
:102FE00064202573207768656E20617474656D7048
:102FF00074696E6720746F2073657420424C455F5E
:10300000434F4D4D4F4E5F4346475F56535F5555B7
:1030100049442E0073645F626C655F6366675F732B
:10302000657428292072657475726E656420257335
:10303000207768656E20617474656D7074696E6761
:1030400020746F2073657420424C455F474154548F
:10305000535F4346475F415454525F5441425F536C
:10306000495A452E0000000073645F626C655F631F
:1030700066675F73657428292072657475726E6562
:1030800064202573207768656E20617474656D70A7
:1030900074696E6720746F2073657420424C455FBD
:1030A000434F4E4E5F4346475F4741502E0000005E
:1030B00073645F626C655F6366675F73657428291C
:1030C0002072657475726E6564202573207768655B
:1030D0006E20617474656D7074696E6720746F2002
:1030E00073657420424C455F4741505F4346475FDC
:1030F000524F4C455F434F554E542E006E72665FE3
:10310000626C655F6761747400000000626C655FEB
:1031100062617300636C6F636B000000434C4F434C
:103120004B0000004750494F544500005052530097
:10313000554152544500000061746669666F2E6DFA
:103140005F717565756500006E72665F6673746F9A
:10315000726167650000000061746669666F2E6DBC
:103160005F6669666F0000007077725F6D676D74EF
:103170000000000062616C6C6F632E6C6F675F6DA6
:10318000656D706F6F6C0000617070006E72665FCD
:10319000736468006E72665F7364685F626C65007A
:1031A0006E72665F7364685F736F6300F43202006F
:1031B000481B0020640200002095010058330200E3
:1031C000AC1D002094150000D09A0100FC300200D4
:1031D000000003030C310200000000001431020063
:1031E000000000001C310200000000002431020039
:1031F000000000002C31020000000000303102000D
:1032000000000000383102000000000348310200D5
:10321000000003035831020000000003683102007F
:103220000000000074310200000000038831020039
:10323000000003038C3102000000030394310200FC
:1032400000000303A031020000000303081D00205A
:10325000001D0020081D002058260020981D002079
:1032600018000000B5AE01000000000059DA0100AE
:103270001C1E00204DA501002C1E002049AD0100A0
:1032800000000000B9AD010000000000B9AF01006E
:10329000000000002FA90100EC1D002091B00100EA
:1032A000001E00207FDB0100E41E00209DAC010019
:1032B000000000000DE1010000000000651A02009E
:1032C0000000000045E1010000000000B7A501007A
:1032D0002C1E00203DEE010000000000C9EF01009F
:1032E00000000000510E02000000000025E1010076
:1032F000000000000322FFFF141418011A0F041A23
:103300000A040128042D8D02022A18017909390ABC
:1033100001A913881D0240200A1A9044122042403D
:103320000425782902146C2F021A0C041A64041A5A
:1033300014041A24041A1C041A2C041A34041A3C07
:10334000041A44041A4C041A54041A5C0449858370
:08335000D00304492DC3010064
:040000050001920163
:00000001FF
